:10000000F01F0010313500002D3500002D350000A7
:100010002D3500002D3500002D35000000000000BA
:100020000000000000000000000000002D3500006E
:100030002D350000000000002D3500005113000098
:10004000FD100000FD100000FD100000FD1000007C
:10005000FD100000FD100000FD100000FD1000006C
:10006000FD100000FD100000FD100000FD1000005C
:10007000FD10000029350000293500002935000059
:10008000091400002114000039140000511400006C
:100090002935000031150000293500002935000000
:1000A00029350000293500002935000029350000D8
:1000B00029350000293500002935000029350000C8
:1000C00008B500230B60036000F096FD08BD08B57D
:1000D0000A20002101F038F908BD000038B50C4BAA
:1000E0000D1C041C19680B4803F056FA212103F07B
:1000F00053FA011C012001F0D7F9012001F0B4F9F5
:10010000291C201C02F084FD012001F0BDF938BD3E
:1001100078800440001BB70008B50A4B0A481968EC
:1001200003F03AFA212103F037FA011C012001F013
:10013000BBF9012001F098F902F0ECFC012001F07C
:10014000A3F908BD78800440001BB70013B59620C2
:10015000000201F02BFA18480D210C2200F02CFCB3
:1001600000F06AFB15480021032200F099FC00F022
:100170006DFBFFF7D1FF1248124901F0FFFB00248D
:1001800001F0BEFA002802D000F0E0FE00240A20B0
:1001900001F00AF9684601A9FFF792FF009B002BC6
:1001A00003D1094B01349C42EADDFFF7B5FF074854
:1001B00001F0E4FB13BDC046583900006037000071
:1001C0006F3700007A3700006F170000813700009A
:1001D00007B5044B04490093044A054B01F0D9FBD1
:1001E00007BDC0469B3700008C3700007A370000FF
:1001F0009537000070B50D1C161C041C00F01CFB8C
:100200000B480D210C2200F0D7FB281CA1B20022C4
:1002100000F046FC07480321062200F0CDFB301C0D
:100220000121092200F03CFC00F010FB70BDC0462B
:10023000583900001338000038B50D1C041C00F0BC
:10024000DAFA2A1C0120211CFFF7D4FF034B0022FD
:100250005A60034A943212689A6038BD281300101D
:100260008C04001010B588B0041C6846FFF7B0FF7E
:1002700069466A46201CFFF7BDFF08B010BD0000AC
:1002800073B518200021FFF729FF00243B4E012001
:1002900001F0FAF83A4D9835002C01D0002000E02A
:1002A0000620012101F050F8684601A9FFF708FF78
:1002B000009B002B21D1002CF0D12B68002B0DD0FE
:1002C000304B00941A6811321A6004E002F0CCFB43
:1002D000009B01330093009B102BF7DD2A4BF6188F
:1002E000DED518200021FFF7F9FE254B94331C685A
:1002F00063425C4100F074FACEE7002C03D0182B67
:10030000C5D100F0ABFA009B182B1BD1019BC22B6F
:1003100008D11E4B1A6801321A60022A0BD1002242
:100320001A6008E0832B06D10020FFF79BFFFFF740
:10033000F3FEFFF7CCFE019B732B01D1FFF706FF05
:1003400000230193124B1348196803F025F921216A
:1003500003F022F9011C012001F0A6F8012001F0B0
:1003600083F80098019902F053FC054B94331B6805
:10037000002B8AD100F034FA012487E720BF020065
:100380008C040010C00200100CFEFFFF7001001072
:1003900078800440001BB70013B501F069FB00F042
:1003A000F7FB00F05BFA00F0DDFD3C24201CFFF7BA
:1003B00059FF013C1E2000F0F7FF022CF6D102F09D
:1003C00075FA1E2300930F2301930E480E4B0F491D
:1003D0000F4A02F025FB00200421012200F0DEFD7F
:1003E0000020021C042100F027FE0020052101222C
:1003F00000F0D4FD00200521021C00F01DFEFFF7D7
:100400003FFFC046F5340000C0020010C1000000EC
:100410003902000000B500E001300378202BFBD04A
:1004200000BD00B5031C303BDAB2092A01D8181C04
:1004300008E020231843031C613B5738052B01D9E2
:100440000120404200BD70B50E1CFFF7E3FF002500
:10045000041C06E0FFF7E5FF002805DB2D0105433E
:10046000013420780028F5D13560201C70BD0000D3
:1004700070B5054E051C0E24013C295D301C01F0B1
:100480007DFA002CF8D170BD9E37000000B50E2318
:10049000013BC25C002A03D1002BF9D1012000E00E
:1004A000002000BDF8B500240E2703231C4221D1F3
:1004B0003E1C66432B4D7019FFF7E8FF002815D04E
:1004C000601C78434019FFF7E1FF00280ED0301C74
:1004D0001C304019FFF7DAFF002807D02A367019C0
:1004E000FFF7D4FF002801D004340DE01E48211C82
:1004F00001F044FA381C60431A4B0134C018FFF76E
:10050000B7FF1A4801F03AFAFF2CCEDD184801F087
:1005100035FA184C201CFFF7ABFF174D4221281C61
:1005200001F02CFA201C0E30FFF7A2FF4321281CFB
:1005300001F024FA201C1C30FFF79AFF0F4801F04D
:100540001DFA201C2A30FFF793FF281C4E2101F0D2
:1005500015FA201C3830FFF78BFF616D084801F059
:100560000DFAF8BD28050010A1370000397B000006
:10057000AA3700008C040010B0370000B737000025
:10058000BD37000070B50E1CFFF744FF0D25041C9D
:100590002078FFF746FF002807DB01347055013D46
:1005A000F6D2201CFFF736FF00E0002070BD0000EF
:1005B00073B5394D08682B78002B06D1374801F008
:1005C000DDF902F073F9012342E00378412B1BD1DE
:1005D000334C0230211CFFF7D5FF002851D003789F
:1005E000422B4ED1211C02300E31FFF7CBFF0028E9
:1005F00047D00378432B44D1211C02301C31FFF734
:10060000C1FF002846D13CE04D2B23D1254C0230C0
:10061000211CFFF7B7FF002833D003784E2B30D1D1
:10062000211C02300E31FFF7ADFF002829D00378DE
:10063000472B26D1023001A9FFF705FF019B002BB4
:100640001FDB2A3C63651848184901F097F900231D
:100650002B701FE001A9FFF7F6FE0378202B01D0D5
:10066000002B0ED1124E00240E250199611869430A
:100670008919FFF787FF002803D00134042CF4D137
:1006800008E002F013F908480A4901F077F9024B33
:1006900000221A7073BDC04698020010C9370000CE
:1006A0008C040010B6040010DF370000E9370000AA
:1006B00028050010EC37000037B54C6824E0201CFA
:1006C000FFF7A8FE01A9FFF7BEFE019B041C002B4B
:1006D0001DD0D8B2FF2B09DD00F0FCF9051C0198F4
:1006E0000012C0B200F0F6F9019003E000F0F2F958
:1006F000002501900198002802D0291CFFF7EEFC8C
:1007000023785A1E9341E4182378002BD7D137BDA4
:1007100008B5064A012113784B40137001D00449F3
:1007200000E00449044801F029F908BD79030010EC
:10073000F3370000FB3700000438000070B5051CDB
:1007400001200821021C00F077FC0724012601206B
:100750000821002200F070FC2A1C224132400020B7
:10076000022100F069FC01200821021C00F064FC59
:10077000013CECD270BD10B50021041C0A1C022003
:1007800000F05AFC201CFFF7D9FF10BDF7B501237C
:1007900000930023019372B66C46061C02AF01CC95
:1007A00050235B421843C0B2FFF7E5FF0020FFF77C
:1007B000E2FF1020FFF7DFFFE020FFF7DCFF00255E
:1007C00002200021012200F037FC705D0135FFF7A7
:1007D000B5FF842DF4D18436BC42E0D162B6F7BDBA
:1007E00008B5AC20FFF7C7FFAE20FFF7C4FFA52078
:1007F000FFF7C1FF08BD08B5AF20FFF7BCFFA4207D
:10080000FFF7B9FF08BD08B5AE20FFF7B4FF08BD7C
:1008100010B5041CF820FFF7AEFF201CFFF7ABFF5C
:1008200010BD10B5041C8120FFF7A5FF3F2020401C
:10083000FFF7A1FF10BD000008B584220248002187
:10084000520001F0D3F808BD8103001008B502483A
:10085000FFF79CFF08BDC0468103001008B50120CA
:10086000021C082100F09AFB0120021C082100F064
:10087000E3FB00200221012200F090FB0020022176
:10088000012200F0D9FB02200021012200F086FBAA
:1008900002200021012200F0CFFB022006210122CC
:1008A00000F07CFB02200621012200F0C5FB0320A2
:1008B000011C012200F072FB0320011C012200F048
:1008C000BBFB0320011C002200F0B6FB0220062126
:1008D000002200F0B1FB06210122022000F0ACFB57
:1008E000FFF7AAFFFFF7B2FFA220FFF744FFA02007
:1008F000FFF741FFC020FFF73EFF0020FFF788FF12
:100900000A2000F051FD4020FFF735FF2C20FFF7B3
:1009100032FF322000F048FD2E20FFF72CFF32205E
:1009200000F042FD2F20FFF726FF0A2000F03CFDDB
:100930002520FFF720FFAF20FFF71DFFA420FFF7C2
:100940001AFF0020FFF76DFF08BD000000B50F295A
:100950000ED883280CD8CB08842253430722C01812
:100960001140044B80220A41111C1A5C1143195496
:1009700000BDC04681030010F0B55B18DBB216E085
:100980008425CC086C4307270F40802504193D417E
:10099000EFB2A6189C4605E0064BE5182B7801340B
:1009A0003B432B70B442F7DB01316346C9B2994235
:1009B000E6D3F0BD8103001000B5084B1860084B6A
:1009C0001970084B20211A70074B1970074BD1087A
:1009D0001970500701D00131197000BD7C0300105F
:1009E000890400108B0400108A040010800300109A
:1009F000F0B5284B89B01B780024C01A264B06920C
:100A000005911B68221C04E002310C190132A4B2CA
:100A1000D2B2195D8242F7DB1B195B780391029316
:100A200000222CE000994B4303999A198A4214DA68
:100A3000194A0025126892191219D3189B78049349
:100A40000123049AAB40134204D07919C9B2079824
:100A5000FFF77CFF0135082DF2D101360837F6B2D9
:100A6000FFB206E00099059A069F8B18DBB20026BC
:100A700007930A490B789E42D4D3019A013201921E
:100A80006B461B79029900938B42EBD309B0081C8B
:100A9000F0BDC0468A0400107C03001080030010E3
:100AA000F7B5171C061C0D1C00F0C0FF80B20190AA
:100AB0000024FFB208E0305DE9B23A1CFFF798FF6E
:100AC00001302D18ADB20134019AA3B29342F2D392
:100AD000F7BD000000B50F23020918408000031F76
:100AE00000D52833002B0EDB511E032088428041A5
:100AF0004042002807D1242B06DC04218A1A03492E
:100B0000CB18985C00E0002000BDC0465B3D0000B3
:100B100010B5041C211C144800F0B2FA211C134823
:100B200000F0AEFA211C124800F0AAFA211C11486C
:100B300000F0A6FA211C104800F0A2FA211C0F4870
:100B400000F09EFA211C0E4800F09AFA211C0D4874
:100B500000F096FA211C0C4800F092FA0B48211C78
:100B600000F08EFA10BDC0462040044024400440EE
:100B7000284004402C400440384004403C4004409D
:100B80004040044044400440484004404C4004403D
:100B9000F8B51020FFF7BCFF094C271C1437257847
:100BA0006678281C311C002200F0F8F90234281C59
:100BB000311C012200F040FABC42F0D1F8BDC04621
:100BC000833D0000F8B50B4C271C14372578667858
:100BD000281C311C012200F0E1F90234281C311CD0
:100BE000002200F029FABC42F0D10020FFF790FF6C
:100BF000F8BDC046833D0000F0B589B000240490E4
:100C00000591FFF7C5FF02200721012206940794F2
:100C100000F0C4F902200721221C00F00DFA201C6C
:100C20000B2100F0DFF9A04202D118230693012422
:100C30000021264D03916A782F78111C0192381CEF
:100C4000012200F0ABF9381C0199002200F0F4F900
:100C500003231F4E029314E03078717800F0C2F93C
:100C6000002807D103991B4AA3008A5C1833694600
:100C70005A500134029A039B013A013302920393C2
:100C8000023EE30F00210122A2424B41DBB28B4224
:100C900002D0029B8B42DFDA381C0199002200F05F
:100CA0007DF90199381C012200F0C6F90A49023584
:100CB0008D42C0D1201E06D0069B049A0599136070
:100CC000079B01200B6009B0F0BDC046833D0000CA
:100CD000593D00005B3D0000973D000000B50A4B08
:100CE00000211960094B01221A6019601A60196805
:100CF0001142FCD0064B01221A60064B8022196873
:100D000052020A431A6000BD70800440748004409F
:100D1000788004408080044008B500F031F90C4B25
:100D200003201A68120B12031A600A4B1A68120B7E
:100D300012031A60084B1A68120B12031A60074B51
:100D40001A68120B12031A60FFF7C8FF08BDC046ED
:100D5000008000500080015000800250008003504D
:100D600070B5124A1249134800F008FE124C13489D
:100D7000211C00F003FE201C00F000FE104E114D5F
:100D800000242B196159DA68301C0B4B143400F025
:100D9000F5FD642CF5D10C4800F0F0FD00F020FBCF
:100DA000011C0A4800F0EAFD70BDC04695370000FE
:100DB0007A370000973D0000093E0000AB3D00007F
:100DC000C43D000000000010CF3D0000F63D0000D3
:100DD000F0B53C4B8BB01D78002D3AD03A4B0290C9
:100DE0001B6801209B685DE001342378202BFBD039
:100DF000002B3AD0B30008336A469C500136FF2DD1
:100E000001D135E001342378202B01D0002BF9D11A
:100E1000202B02D1002323700134012E1BD12A4F35
:100E20002A4B06223B6001923D1C09E02B68029888
:100E3000196800F00EFE002808D02B6814332B60D0
:100E4000019B013B0193002BF0D132E03B681D79FF
:100E500001E0041C2E1C2378002B06D0002307225F
:100E6000B2425B41DBB2002BBFD1002E1CD000E0B0
:100E70000025154C022E05D10398154900F0E9FD17
:100E8000002801D0AE420AD823681248D96800F081
:100E900075FD23681048196900F070FD04E02368AF
:100EA000F0B29B6802A99847064B1B78002B07D12C
:100EB00003E00198011CFFF753FF084800F05EFDB6
:100EC0000BB0F0BD98020010A0020010000000104E
:100ED000033E0000053E0000E43700000C3E000029
:100EE00038B5041C154D0A2808D002D808281CD192
:100EF00010E00D2802D07F2817D10BE02B680022CC
:100F00001A700F4800F03AFD0E4C201CFFF760FFEE
:100F10002C6012E02A680B4B9A420ED90A48211C19
:100F200000F02CFD2B68013B06E00748211C00F077
:100F300025FD2B681C7001332B6038BD9C0200100E
:100F4000093E000098010010183E000008B503E0BB
:100F500000F0B4FBFFF7C4FF00F0D2FB0028F7D18C
:100F600008BD000008B5034A034B04481A6000F0AE
:100F700005FD08BD980100109C0200100C3E000009
:100F8000044B40211A680A431A60034B01221A706D
:100F90007047C04680800440A402001070B50E4B1C
:100FA000061C1B780D1C141C002B01D1FFF7E8FF59
:100FB000013E022E03D8094BB600F35800E0084B5F
:100FC0001A68012C03D1AC4014431C6003E00124D7
:100FD000AC40A2431A6070BDA4020010843E000021
:100FE0000080005038B50F4B051C1B780C1C002BE3
:100FF00001D1FFF7C5FF0020032D11D8281C0123C4
:1010000002F0B6FA02040608074A04E0074A02E0C2
:10101000074A00E0074A1068A3401840431E984161
:1010200038BDC046A4020010FC3F0050FC3F0150F8
:10103000FC3F0250FC3F035070B50E4B061C1B7862
:101040000D1C141C002B01D1FFF79AFF013E022E4C
:1010500003D8094BB600F35800E0084B1A68012C7E
:1010600003D1AC4014431C6003E00124AC40A24314
:101070001A6070BDA4020010903E0000FC3F0050BA
:1010800038B5084B041C1B780D1C002B01D1FFF751
:1010900077FF236818229343236023681D4325604C
:1010A00038BDC046A40200101F2342091840012386
:1010B0008340181C014B9200D050704700E100E0C3
:1010C000054B3F221A60054B01221A60044B402158
:1010D0001A688A431A60704724800440D88004400C
:1010E0003882044008B5044B40211A688A431A60CC
:1010F000FFF7E6FF08BDC0463882044008B503206C
:10110000FFF7ECFD094B012252421A60084A1268AF
:10111000002A00D01A60074B1A6801321A60064A8A
:1011200000231360054A1360C04608BD08820440CE
:101130000C820440A802001004C000403CC00040E3
:1011400008B5FFF73FFD0A480021FFF799FF09485E
:101150000021FFF795FF08480021FFF791FF07489E
:101160000021FFF78DFF06480021FFF789FF08BD2A
:101170000840044000400440AC4004401440044097
:101180001C400440F7B50190FFF7DAFF574B019977
:101190001A68574B1A60002901D0564B00E0564B95
:1011A000564A04211360564B564C1A68564D0A4352
:1011B0001A60019A002A54D0544B0027544E1F60E5
:1011C000544B301C1F60391CFFF75AFF381C092193
:1011D0003A1CFFF7E3FE381C09213A1CFFF72CFFED
:1011E0004D4B802219680320114319603368072191
:1011F0008B433360336802210B43019933604B000A
:101200005B1899015B1801999B005B1843490B60BF
:10121000434B196801431960424B43491868014028
:101220001960196809200A431A60FFF73DFF226818
:1012300080239B001A43226001213C4A49421160ED
:101240002A68324913432B60394B02221A60394B0A
:1012500001221A601F601A6018681042FCD0012336
:101260000B600720FFF720FF0820FFF71DFF0A2073
:10127000FFF71AFF0C20FFF717FF0B20FFF714FFF3
:10128000236880229343236022682B4B1340236002
:1012900022682A4B134023602268294B13402360A5
:1012A0002268284B13402360019B002B03D10122AD
:1012B0001E4B52421A602B68802213432B602A680F
:1012C00080235B0013432B602A688023DB001343D9
:1012D0002B602A6880235B0113432B602A688023DC
:1012E0001B0113432B6030BFF7BDC046388204405A
:1012F00034820440BF180000FF1800003082044010
:1013000010ED00E0008204400482044004C000406C
:1013100064400440044001408080044018C0004004
:1013200014C000403CC000400FF0FFFF08820440A2
:101330007080044074800440FFFEFFFFFFFBFFFF4E
:10134000FFEFFFFFFFF7FFFF08B5FFF71BFF08BD2B
:1013500000B5064B1A6801321A601B68013303D1CD
:10136000034B1A6801321A6000BDC046B00200107B
:10137000AC02001000B5074B98420AD8064A002379
:101380001360064A01381060054A1360054B0722B6
:101390001A6000BDFFFFFF00B002001014E000E083
:1013A00018E000E010E000E000B50C4A13680028E7
:1013B00000D10120C1438B4204D809E01168814269
:1013C000FCD301E0591C081811689942F6D203E0D9
:1013D0001168C91A8142FBD300BDC046B00200109B
:1013E00010B5064BFA211868054B89001C6802F0FD
:1013F000D3F8044B5C43201810BDC046B002001067
:10140000AC02001037894100034B01221A60034BE4
:101410001A6801321A60704700C00040B402001020
:10142000034B01221A60034B1A6801321A6070479D
:1014300000000140B8020010034B01221A60034B68
:101440001A6801321A60704700400140BC02001067
:10145000034B01221A60034B1A6801321A6070476D
:1014600000800140C002001000B5002803D1044BE9
:1014700001221A6003E0012801D1024B186000BD6F
:10148000044001400480014000B5002802D1044B13
:10149000186004E0012802D1024B00221A6000BD4E
:1014A000044001400480014010B5041C002906D10D
:1014B000164B96201968C00002F06EF8011C002C33
:1014C0000FD1134B80221868920002431A60114B0F
:1014D00003221C60104B1960104B1A608022D2024C
:1014E00011E0012C11D10A4B80221868D20002436E
:1014F0001A600B4B00221A600A4B032219600A4B38
:101500001A6080221203094B1A6010BD78800440D3
:1015100080800440BC02001018400140144001408B
:10152000C0020010188001401480014000E100E07A
:1015300008B5184B1A680E231340062B0DD1164B15
:101540009E221B68DBB2134204D0144A5360144B32
:101550001B681EE0D9071CD501E0042B05D1104BF8
:101560001868C0B200F0BBF813E00C2B06D10B4B8F
:101570008022596852000A435A600AE0022B08D1BF
:10158000054B1A68054B910601D5002200E00122A7
:101590009A6008BD0880004014800040C40200101A
:1015A0000080004000487047C402001070B52B4C0A
:1015B0002B4B80229203DA6700219022061C201C0C
:1015C00000F014FA0023A36000F072F8254B072501
:1015D0001A68254CAA431A60196801221143196040
:1015E000224B1968A9431960196811431960204BEF
:1015F000802118684901014319601E4B1E481A607A
:101600008322226019681D4B1B68584301F0C4FFF8
:10161000311C000901F0C0FF1949030A194A0B6087
:10162000C0B2032310602360174B1D60174B18686E
:1016300060201C680440602CFBD101E0146800E0CD
:1016400001201C680442F9D1044B01221A70104B8E
:10165000802292031A6005230B6070BDC402001043
:1016600004E100E0A44004400C800040A840044095
:101670008080044098800440001BB70078800440BC
:10168000048000400080004008800040148000403A
:1016900000E100E000B5044A202311681942FCD0A3
:1016A000024B186000BDC04614800040008000401E
:1016B00008B5FFF777FF0023437308BD08B5FFF7B0
:1016C00071FFC27B031C8218107CDA7B7F21013200
:1016D0000A40DA735A7B013AD2B25A7308BD10B588
:1016E000041CFFF75FFF837B7F22C3181C74837B7E
:1016F000013313408373437B0133DBB2437310BD6B
:1017000008B5FFF74FFF407B431E984108BD30B539
:10171000002402E00570013401301D5D002DF9D177
:10172000121B131C02E00170013B0130002BFADC9C
:10173000D043C0170240A01830BDF8B5051C0F1CDF
:101740001E1C541E092B01D800240FE0181C0A216E
:1017500001F022FF221C031C391C281CFFF7EDFF9F
:10176000041C2D1805E02F7001340135013A002AC0
:10177000F9DC301C0A2101F053FF30312970601C64
:10178000F8BDF8B50C1CD9175F18061C4F40551E44
:10179000092F12D9381C0A21002B03DA01F0FCFEB4
:1017A000434202E001F0F8FE031C211C2A1C301CFD
:1017B000FFF7E7FF041C351813E0002B00DA951E35
:1017C000002201E0B4540132A91A0029FADCEC43EA
:1017D000E4172C403519002B03DA2D232B7001342C
:1017E0000135381C0A2101F01BFF30312970601CC3
:1017F000F8BD73B5069E041C1D1C3009531E00283D
:101800000AD000901A1C201C2B1CFFF7F2FF241892
:1018100005E0217001300134013A002AF9DC0F2380
:101820001E40092E01D8303604E0002D01D0373695
:1018300000E057362670013076BDF0B585B0041C47
:101840000F1C002801D00021017000256BE0252924
:1018500003D021700132013405E05178252904D1EB
:1018600021700232013401355DE0302903D00132AC
:101870000292202101E002320292029E9C463278BE
:101880002D3A50424241B6180296002205E00A2342
:101890005A438218303AD2B201363078031C303BBA
:1018A000092BF4D90296AE186346BE4201D97A1BC1
:1018B000D2B269280ED006D863282CD0642809D06B
:1018C00058283ED119E075280AD078280FD07328FF
:1018D00037D11AE01E1D201C1B68FFF752FF04E0E1
:1018E0001E1D201C1B68FFF728FF331C17E01E1D60
:1018F0001B68201C0093002304E01E1D1B68201C95
:1019000000930123FFF775FFEFE71E1D201C1B68E6
:10191000FFF7FDFEE9E71A68012022700433029AFE
:10192000241801322D181178BD4201D200298ED120
:101930000023BD4201D2237005E0013C2370013D2C
:1019400001E001256D4205B0281CF0BD10B50C1C4E
:10195000131C6421221CFFF770FF10BD00B5031C8F
:101960009BB00A1C01A8191CFFF7F0FF632800DDDB
:10197000FEE701A800F09CF81BB000BD0FB407B54E
:1019800004A901C90191FFF7E9FF03B008BC04B045
:1019900018470EB403B503AA02CA0192FFF7D6FF97
:1019A00002B008BC03B0184770B50323041C1842EA
:1019B00005D10D1C041C194201D1934201D300230F
:1019C00011E0131C40CD043B40C4032BFAD8141F74
:1019D000A4080134A400032309191A400419EEE7EE
:1019E000CD5CE55401339342FAD170BD30B50B04A0
:1019F0000D061D430D430B021D430323041C93429C
:101A00000DD218420BD1131C043B20C4032BFBD86E
:101A1000141FA4080134A40003231A40041900234E
:101A200001E0E15401339342FBD130BD00B5002306
:101A300000E00133C25C002AFBD1181C00BD00B5D8
:101A4000031C01E0013101330A781A70002AF9D130
:101A500000BD00B502E00130002B06D00A78037803
:101A600001319342F7D0981A00E0181C00BD000025
:101A700008B5FFF751F90B48FFF77CFCFFF780FA38
:101A8000FFF730FB96200002FFF790FDFEF7E6FE21
:101A9000FEF7D2FE044A0548111CFFF76FFFFFF75F
:101AA00061FA08BDE02E0000093E00009C3E0000E7
:101AB00010B5041C02E00134FFF7ECFD207800288B
:101AC000F9D110BD00B50B4B984201DD0A4BC0188F
:101AD0000A4A8310D35C03220240082152008A1A6A
:101AE00093401A1CC0239B001A40054B1B5C101C22
:101AF000184300BDFF17000000F8FFFFCA3E0000BA
:101B0000CA4A000008B54018511A013101F0F4FD2D
:101B100008BD08B5801889189A1A0132FFF744FFEA
:101B200008BD000030B5B14B87B0D96EB04D4A1E2C
:101B300091416A46D175A96A1A1CC806400F01383E
:101B4000062807D801F014FD040C1F1217191C00F9
:101B5000022409E05A6E16329200D3581C1C15E07C
:101B60005B6E16339B00D45800230FE09B6DD46D41
:101B7000A3420ADC0AE0022403E00C24032305E06C
:101B80000D24231C02E00D24EEE70D242C614811E6
:101B90001F2800D922E16A461732944901F0F2FC6D
:101BA0002000220028002A002D002F0038004000CD
:101BB0004400490051005F0067006F007700850016
:101BC0009300A200B400C300D500D300E300E600F8
:101BD000E900F100010105010F01110113011901D3
:101BE000081C00E08348191C221CFFF78BFFF5E05E
:101BF0008148F8E70A1C0E3203E07E4809E00A1C1F
:101C00001C32081C111C1A1C231C01F003F9E5E00E
:101C10007948011C0E391A1C231CFFF77AFFDDE0FE
:101C20007448011C0E31EEE70A1C1C32081C111C02
:101C3000F1E70A6E1020002A00D00A200A1C0E329A
:101C400006E00A6E1020002A00D00A200A1C1C326E
:101C500000946C46173402900194081C51E0012056
:101C60001070086E1022002844D00A2242E00A6E4A
:101C70001020002A00D00A200A1C0E320EE001209B
:101C80001070086E1022002855D00A2253E00A6E08
:101C90001020002A00D00A200A1C1C3200946C4636
:101CA000173402900194081C78E00A6E1021002A73
:101CB00000D00A21504A68461730019002910094E2
:101CC000101C111C1DE00A6E1020002A00D00A20F2
:101CD000494A00946C46111C173402901C39019437
:101CE000101C0EE0096E012010701022002900D097
:101CF0000A22414968461730019002920094081C5C
:101D0000002201F091F869E00A6E1020002A00D04C
:101D10000A20394A00946C46111C173402901C3971
:101D20000194101C3AE0096E012010701022002965
:101D300000D00A2230496846173001900292009480
:101D4000081C00222AE0012010700A6E1021002ACF
:101D500000D00A21284A6846173001900291009469
:101D6000101C00211AE0009222481CE00092224838
:101D700019E00A6E1020002A00D00A200A1C1C322A
:101D800006E00A6E1020002A00D00A200A1C0E323B
:101D900000946C46173402900194002001F06DF815
:101DA0001CE00092081C002104E00D1C1C35081CDE
:101DB0000092291C1A1C231C01F0BAF80EE0081C22
:101DC00002E00C4800E00C48191C221C01F0C9F884
:101DD00004E0081C221C191C01F0CEF86B46DA7DC9
:101DE000024B07B00120DA6630BDC0468C040010FB
:101DF000281300109A040010A804001010B506491A
:101E00000B1C88331A68141C1E34A4006050013265
:101E100003210A401A6010BD8C040010054B0320FA
:101E2000191C88310A68013A02400A601E32920089
:101E3000D05870478C040010F8B5114D2C1C8C3410
:101E400020680130FFF73EFE0E4B0122D8629F6AE8
:101E5000AB6E061C02409A4210D1830703D420685F
:101E60000230FFF7CBFFFF239B001E40B601BF10DF
:101E7000044B8C35374301222F60DA600220F8BD15
:101E80008C0400102813001030B50C4B0C489A6AD3
:101E9000031C8C331C68D3059B0E910500D5403B79
:101EA000856E921001210A40AA4204D1E3188C30B9
:101EB0000360024BD960012030BDC04628130010DA
:101EC0008C04001008B5084B5A1CD07F9A1CD27F96
:101ED000000112021043DA7F0333DB7F10431B0340
:101EE0001843FFF78BFF08BD8C04001038B5FFF7CF
:101EF00095FF064903230F22051C5C18154001338A
:101F000025770011072BF7D138BDC0468C0400108F
:101F100008B5FFF783FF034B01228C331860024B97
:101F2000DA6008BD8C0400102813001010B5064CB0
:101F3000A36E002B06D0FFF771FF044B8C340122F7
:101F40002060DA6010BDC0468C0400102813001019
:101F500010B5064CA36E002B06D1FFF75FFF044BB4
:101F60008C3401222060DA6010BDC0468C04001061
:101F70002813001008B5124B1B68002B00D098479F
:101F8000104B5A69002A15DD012A07D1DA69002AA7
:101F900004D09A610022DA610A225A615B69032245
:101FA000191C91430A1E02D0074A0121D166054A35
:101FB000013B5361044B90331A68024B5A6208BDCF
:101FC00054030010281300108C04001000B5064BB9
:101FD0005A69002A07DD9A690F21044B1140D9770D
:101FE00012110133DA7700BD281300108C040010A1
:101FF000044B597F9A7F090112020A43197F0A4351
:102000005A6770478C04001030B50B1C093B012B3C
:102010000FD8084A00239C18257FC45CA54205D030
:10202000054B08395A681143596002E001330E2B01
:10203000F1D130BD8C0400102813001000B5082920
:102040000DD0192911D1427808231A4202D000225A
:10205000027002E00F2303700723437005E00023A2
:102060001A1CC25401330E2BFBD100BD10B50E4B10
:10207000596F002802D00F22914301430E244C4394
:1020800059679C33E418094B1B68292B02D0201C8C
:10209000FFF7D4FF044A0023E05C99180133087766
:1020A0000E2BF9D110BDC0468C040010281300106F
:1020B00070B5124B0F225C6F944304435C67104B66
:1020C0001B68292B01D0082C17D00E2565430D4E17
:1020D000211CAD19281CFFF797FF9C3E00239A197D
:1020E000127FEA5401330E2BF9D1054B1B68292BC3
:1020F00003D0281C211CFFF7A1FF70BD8C04001029
:10210000281300102805001038B5104B104D1B681F
:10211000292B02D06B6F082B17D0696F0E244C430C
:102120009C356419201CFFF76FFF9C3D00235A1952
:10213000127FE25401330E2BF9D1044B1B68292B7B
:1021400003D0696F201CFFF779FF38BD28130010FA
:102150008C04001010B50D4C631CD87FA31CDB7FD2
:1021600000011B021843E37F1843E31CDB7F1B03C2
:102170001843FFF7A7FC0F23021C1A402277021115
:10218000134000126377A07710BDC0468C04001086
:10219000044B5A6E16329200D258121A51424A41DA
:1021A000DA6670478C04001000B5064B5A6E163282
:1021B0009200D1580139D150002901DA0D21D150B6
:1021C00000BDC0468C04001000B5064B5A6E163296
:1021D0009200D1580131D1500E2901D10021D150A6
:1021E00000BDC0468C04001000B5094B5A6E163273
:1021F0009200D2580D2A03D11A1C2932127805E018
:102200009A18507F117F0001021C0A435A6500BDD5
:102210008C04001010B5084B0F245A6E1632920031
:10222000D1585A6D58181440013104770D2902DC39
:102230005B1812111A7710BD8C04001030B50F4BCB
:102240005A6E596D16329200D2580D2A07D11C1CB5
:1022500029342478F02008402043586507E0981876
:10226000447F057F24012C435C650B114377034BAE
:102270009A180F231940117730BDC0468C04001006
:1022800008B504480022011C1C390D23FFF741FC4E
:1022900008BDC046C404001008B504480022011C53
:1022A0001C310D23FFF735FC08BDC046A804001003
:1022B00008B504480022011C1C310D2300F0AAFDC2
:1022C00008BDC046A804001008B504480022011C3F
:1022D0000E390D23FFF71DFC08BDC046B6040010E3
:1022E00008B504480022011C0E310D23FFF711FC34
:1022F00008BDC046A804001008B504480022011C0F
:102300000E310D2300F086FD08BDC046A804001064
:102310000C4A0023111C46310B70111C47310B7005
:10232000111C48310B70111C49310B70111C4A31C2
:102330000B70111C4B310B70111C4C314D320B705A
:10234000137070478C04001000B5074A011C042369
:1023500000208A1804E0D11846310978400008436B
:10236000013BF8D200BDC0468C04001030B5074ACE
:1023700000238918012206E0CC18051C46341540BC
:10238000257040100133042BF6D130BD8C040010B1
:1023900038B50020FFF7D8FF084C051C0021207F2E
:1023A000FFF7E4FF25770420FFF7CEFF0421051C8B
:1023B000607FFFF7DBFF657738BDC0468C040010F7
:1023C00010B50020FFF7C0FF034C20770420FFF773
:1023D000BBFF607710BDC0468C04001010B5054CE3
:1023E0000021207FFFF7C2FF607F0421FFF7BEFFBF
:1023F00010BDC0468C04001010B5094C231C8C3352
:1024000018680130FFF75EFB064B021CD8620F23F1
:102410001A4022770211134000126377A07710BD93
:102420008C0400102813001010B5094C0021201C4A
:102430000D22FFF767FB201C0E3000210D22FFF755
:1024400061FB201C1C3000210D22FFF75BFB10BD3F
:102450008C04001010B50C4B00211A1C187F1C783E
:1024600001312043187701330E29F7D1936E002BE9
:1024700008D0064B1B690D2B04D1137F111C293189
:102480000B70537310BDC0468C040010281300104D
:1024900010B50C4B00211A1C1C7F1878013120400C
:1024A000187701330E29F7D1936E002B08D0064B15
:1024B0001B690D2B04D1137F111C29310B70537331
:1024C00010BDC0468C040010281300107FB50023F7
:1024D0000C4A0D251C1C1118097F01306E469955B8
:1024E000C60F8542664176420133111C30400E2BE7
:1024F000F1D100236C46185DCA18013310770E2BFA
:10250000F8D17FBD8C04001010B5074B5A6E1632FF
:102510009200D1585C1801392077D150002901DA96
:102520000D21D15010BDC0468C040010034A002379
:10253000111C943198320B60136070478C040010AA
:10254000034B012194331A684A401A607047C04611
:102550008C040010044A002313678C321360034B71
:102560000122DA607047C0468C0400102813001066
:1025700008B59A4B0F20996A994A8B101840891117
:10258000013852560E2800D9C1E000F0F1FF0811C1
:102590001A2327C02EC0C037C0C0C03B3F00002A4E
:1025A00000DAB4E08F4B9A18403200239371A9E00F
:1025B000002A00DAABE08B4B01209A184032907170
:1025C000A4E0002A00DAA2E0864B9A184032927901
:1025D000DA6697E0081CFFF797FF93E0002A00DA1D
:1025E00095E0101CFFF7D4FD8CE0002A00DA8EE0A5
:1025F0007C4B596E16318900CA5083E0081CFFF7E6
:1026000057FD7FE0081CFFF731FD7BE0002A00DA70
:102610007DE0101CFFF75AFF74E0724B01209833E5
:10262000186073E0FFF7E0FD6CE0FFF793FF69E0EF
:10263000FFF726FE66E0FFF7EDFD63E0694B002241
:102640005A665FE0FFF728FE5CE0FFF7F7FD59E010
:10265000644B0120586659E0FFF72AFE52E0FFF76D
:10266000CBFE022052E0FFF72FFE4BE0FFF72AFCE3
:1026700048E0FFF735FE45E0FFF7D6FE42E0FFF702
:1026800035FC3FE0FFF738FE3CE0FFF79FFC39E008
:10269000544B00221A6635E0FFF7AAFC32E0514B9A
:1026A0000120186632E0FFF741FF2BE0FFF72CFD19
:1026B00028E0FFF745FF25E0FFF74CFD22E0FFF79C
:1026C0008DFE1FE0FFF732FC1CE0FFF7C3FE19E0B0
:1026D000FFF776FE16E0FFF73BFC13E0FFF7D8FEAE
:1026E00010E0FFF715FE0DE0FFF744FC0AE0FFF7EE
:1026F0005BFD07E0FFF74CFE04E0FFF765FD01E03E
:10270000FFF706FC012001E00120404208BD982BA4
:10271000BED03EDC382B9BD01DDC1C2B00D187E7C4
:102720000CDC0C2B00D178E702DC002BEAD0EBE7C5
:10273000162B00D176E7182BE6D176E7282B00D1AF
:102740007CE702DC262BDFD175E72C2B00D179E763
:10275000362BD9D179E7662B00D18AE70CDC4C2BDC
:1027600000D17CE702DC3C2BCED175E7562B00D1A3
:1027700079E75C2BC8D179E76C2B00D17FE702DCCD
:10278000682BC1D178E7762B00D17BE7882BBBD1B2
:102790007BE7E62B00D19BE726DCC82B00D188E73E
:1027A0000CDCA82B00D17AE702DC9C2BACD173E7C0
:1027B000B82B00D177E7BC2BA6D177E7D62B00D179
:1027C0007DE703DCCC2B00D09EE775E7D82B00D14A
:1027D00078E7DC2B00D097E777E7C0462813001096
:1027E000CA7A00008C040010F32B00D17CE70EDCC9
:1027F000EC2B00D172E703DCE82B00D084E76AE71A
:10280000F12B00D16DE7F22B00D07DE77AE7F62BB4
:1028100000D16FE703DCF52B00D075E767E7F72BF6
:1028200000D16AE7F82B00D06EE769E738B5184C9D
:10283000231C8C331868FFF745F9211CE26E903198
:10284000144B0D68A2660022E2660135DA600322AD
:1028500098620D601040251C1C1C022809D0904273
:102860000AD0012802D0FFF783FE07E0FFF7E4FA61
:1028700004E0FFF757F901E0FFF706FB002806DD4B
:10288000E368002B03D18C352B681B182B6038BDF7
:102890008C04001028130010034B0122DA660F226B
:1028A0009A775A771A7770478C04001010B5054C48
:1028B0000549201C00F020FFFFF7EEFF01236366AF
:1028C00010BDC0468C0400109C0E000000B5074BE4
:1028D00000201B680F2B08D1054B1A78824204D1C7
:1028E0001868044B1840431E984100BD6400001056
:1028F0008C04001000FFFF0038B5164B1A1C9832EC
:102900001268002A04D0144B1D6801231D4001E009
:1029100094331D68114CA3689D4202D16268002A5D
:1029200016D0002D02D1002B0AD111E00C4B1B68F0
:10293000002B02D06168281C98470023636006E0E2
:10294000074B1B68002B02D0281C291C9847A56048
:1029500038BDC0468C04001074030010281300100A
:102960006C03001013B5002300930193244B1B68E4
:10297000002B02D0684601A998472249009B08789D
:10298000214A00280CD0002B02D00223137035E01E
:102990001378013BDBB21370002B2FD10B7009E0D1
:1029A000002B0CD11378002B28D0013BDBB2137025
:1029B000002B23D1154A1360154A13601EE01449F9
:1029C0000968581A44426041400010701148446937
:1029D000021C002C04D08B4202D10A2343610DE07B
:1029E00000290BD10A21516101999361D161084AF3
:1029F0001360064B02221960034B1A7013BDC046C8
:102A00005C03001078030010600300105C130010DA
:102A1000581300102813001008B5FFF7A3FF08BDD6
:102A200010B5094C20600948016009490A60094A4B
:102A30001360094B029A1A60084B039A1A60084AFD
:102A4000084B1A6010BDC0466C0300105C030010F8
:102A500068030010640300105803001064000010A5
:102A6000192A00005403001008B5084B084A1968D9
:102A700012688A1A1A6006D5FA2252001A60054BAB
:102A80001A6801321A60FFF737FF08BD68000010AE
:102A90005803001074030010F7B50E1C0E21051C1E
:102AA000019200F029FE1A4B03240C279E420FDDF1
:102AB00009236B7301232B7328E0301C0A2100F0DB
:102AC0000FFE301C29550A2100F0B4FD0134061C0C
:102AD000002E06D0E30F0022A7425341DBB29342FF
:102AE000EBD1019AA31A033B2B70621B2B1C01E054
:102AF000195D5973013BD1180229F9D10F231C1B11
:102B0000002301E0013C2B55032CFBDCF7BDC04644
:102B1000FFC99A3B38B50C4B01221A700B4B0222AD
:102B20001A700B4D0B4C08E01868884208D01B68DF
:102B30002360FFF799FFFFF715FF2B682168024A12
:102B400010780028F0D138BD780300106003001021
:102B500064030010700300104278037812011A43D6
:102B6000C37881781B010B43D01A7047F0B5224A15
:102B7000224B0F1CD45CE8235B00D35C24011C4374
:102B80001F4BE121D35C4900515C1B0185B00B4315
:102B90000293E9235B000390D55C002C02D18024D2
:102BA00007256400174E301CFFF7D6FF0299421C20
:102BB000631A802149000C1B07214D1B0398124901
:102BC00001950094FEF7E5FE00233B704125023E8F
:102BD000381CFEF72BFF3C18301CFFF7BDFF2A1CEA
:102BE000031C0A49201C0135FEF7D3FE023E462D88
:102BF000EED105B0F0BDC0468C040010D10100003C
:102C0000C301000058060010DA7A0000E77A0000DD
:102C100030B5404B404C1A1C9432126891B0A06100
:102C2000E161002A17D118280BD1C32909D13B4AE9
:102C300012680F2A05D1181C38300E21162200F018
:102C4000D5F8A369182B04D1E369332B01D100F027
:102C500077F8FFF721FE0A2363612E4C0123304DE4
:102C600023678C34FFF7E2FD2368AB4218D006DC03
:102C70002C4A934219D02C4A934233D106E02B4A76
:102C8000934208D02A4A93422CD117E0234B1B6869
:102C90000B2B27D10DE0214B1B680C2B22D108E018
:102CA0001E4B1B680F2B1DD103E01C4B1B68102B08
:102CB00018D1FFF721FEFDF70AFA13E0174B1B6846
:102CC0000F2B0FD1684608A9FFF750FF194B1B685F
:102CD000002B02D0684608A998470E4B8C331A681F
:102CE00027321A60144B1A68144B1068196888420E
:102CF00005D012681A60FFF7B7FEFFF733FE054BE9
:102D00001B6F002BAED1FFF7F7FDFFF703FF11B0EC
:102D100030BDC0468C040010281300106400001061
:102D2000790D00006A0C0000130D0000990D0000E1
:102D30003E270000680300106403001070030010B9
:102D400070B5254C23681D68FFF7E4FE23681A68F8
:102D50009542FCD01E68FFF79FFD204B0A22204CB5
:102D60005A6118229A611522DA61231C90330022DD
:102D70001A60FFF791FD012323676436164C194D45
:102D80000AE0FFF753FD23682A681968914203D0CF
:102D90001B682B60FFF768FE23681B689E42F0D11A
:102DA0000F4D18202B1C90331C680021FFF730FFBB
:102DB0000D4B60001968001900F03CFC3835011C0F
:102DC0000422281CFFF768FE044B18229A61002297
:102DD000201CDA6170BDC046640300102813001087
:102DE0008C0400107003001058030010F0B501248B
:102DF0000DE005780B1C254006E0C65CED00770869
:102E00003D43C554351C2540013BF6D5013A002A07
:102E1000EFDCF0BD30B504E0845C8D5C85548C54EF
:102E200001329A42F8DD30BDF7B5099D0AAC26782B
:102E3000089F2C7894461D1C002A0DD118E063468B
:102E40005B5D4A5DD218131901920024B34201DB85
:102E50009B1B012443550135BD42F0DD0AE0CA5CED
:102E600012190024B24201DB921B0124C254013327
:102E7000BB42F4DD099B1C70F7BDF7B5099E0AAC97
:102E80002778089D347800282FD000292AD01E1CCE
:102E90009446002A0ED1013F18E063469B5D8A5D8F
:102EA000D21A131B00240192A34201DADB19012478
:102EB00083550136AE42F0DD37E0CA5C121B0024B8
:102EC000561C01D13A1C0124C2540133AB42F4DD3B
:102ED0002BE0D15C49420C1B211E01D0E1190124D9
:102EE000C1540133AB42F4DD1FE000291BD0181C94
:102EF000002A06D10EE00E5C135C0130F31A1C1B95
:102F0000E40FA842F7DD10E0CA5C0133141B013462
:102F100062425441AB42F7DD07E0D15C01334942E4
:102F20000C1B611E8C41AB42F7DD099A1470F7BD92
:102F300070B5049D01242C70141C002905D10BE0F0
:102F4000065D0A5D96420BD101349C42F8DD05E036
:102F5000815C002904D101329A42F9DD00232B70F3
:102F600070BD00B503E043185B78435401319142D2
:102F7000F9DB0023435400BD00B504E08318013B96
:102F80001B788354013A8A42F8DC0023835400BD45
:102F9000F0B5114B1A785B78825C1A4000D0402261
:102FA0000E4C0F49231C261C04C32C3600221A6029
:102FB00001240A1C123117785578C75D3D4202D0B2
:102FC0001F6827431F60023264008A42F3D1043332
:102FD000B342EBD10020F0BD61010010F0140010ED
:102FE000AD00001030B512234B43334A0131D318E2
:102FF0008A0051181A785C78825C144204D02F4AF7
:103000005F245218947054709A78DC78825C144271
:1030100004D02A4A7C245218533214701A795C79ED
:10302000825C144204D0254A7C245218A3321470C6
:103030009A79DC79825C144207D0204C5F226418B4
:10304000251CA235A1342A7022701A7A5C7A825C1F
:10305000144204D0194A7C245218A03214709A7A6F
:10306000DC7A825C144204D0144A7C245218503218
:1030700014701A7B5C7B825C144207D00F4C5F2279
:103080006418251C523551342A7022709A7BDC7BDF
:10309000825C144204D0094A2E245218A4321470BF
:1030A0001A7C5B7C825C134204D0044B5918F431C7
:1030B00027230B70002030BDAD00001060130010FE
:1030C000F8B52D4C071C0025201C20214F22FEF7AF
:1030D0008DFC002D04D0221C7C2339322370137008
:1030E000231C4F330021013519705034052DEBD1CD
:1030F000214B2D22181C38300270181C37300270FA
:10310000A1209A705A7040005F221A541B481A542A
:10311000A320400019541A4908784978385C0142C4
:1031200004D0191C533152330A701A700024211C28
:10313000381C0134FFF756FF0A2CF8D1114D124EFE
:1031400000242B786A78FB5C1A4201D0315905E0E3
:103150003059FEF76BFC0D49091A0A310C4804344A
:1031600000F0D4FA0235242CEBD10A49084800F0CB
:10317000CDFA0520F8BDC0466013001041010000E3
:10318000610100106C00001080000010630100104D
:10319000A0140010EF7A0000F0B585B00190002770
:1031A000FDF74AFB6A4C3E1C6A4A7542754113683A
:1031B0007D19012B05D168480D210C22FDF7FCFB80
:1031C00002E0002B00D1CDE0002303AA5370236856
:1031D0007F210B405C2B00D198E02ADC382B00D1FA
:1031E0008EE013DC072B6AD006DC022B00D193E0C3
:1031F000062B00D0B6E041E0212B00D184E0232B48
:1032000000D187E01C2B00D0ACE081E04F2B4ED0EA
:1032100007DC3F2B62D0402B62D0392B00D0A1E0DD
:1032200064E0542B76D05B2B3FD0502B00D099E03C
:103230006AE0732B66D010DC662B3AD005DC5E2B7F
:1032400056D0622B00D08DE062E06F2B3BD0712B0B
:1032500052D06D2B00D085E02DE0792B4AD006DCD2
:10326000762B4BD0772B3DD0742B7BD146E07D2B3A
:1032700023D07F2B25D07C2B74D135E031231370E4
:10328000022E4BDD231C083B1B681940542908D033
:10329000032E43D0231C0C3B1A687F231340542B6E
:1032A0003CD14C2203AB1A7038E0322335E0332393
:1032B00033E0342331E035232FE036232DE037236C
:1032C0002BE0382329E039231370062E26DD231F37
:1032D0001B6819404723232920D11EE030231CE01E
:1032E0002D231AE0412318E0422316E0432314E083
:1032F000442312E0452310E046230EE048230CE06F
:103300004C230AE0502308E0522306E04F2304E058
:10331000552302E04E2300E049231370ADB203A809
:10332000291C0022FDF7BCFB23681A0605D5E91D00
:1033300089B20A480022FDF7B3FB2368DA0572D58B
:103340000735A9B206480022FDF7AAFB6BE0C0468C
:10335000F01400107001001058390000443E0000C5
:10336000F77A000023680122134206D0A818C0B2E1
:10337000002107220223FDF7FFFA236802221342ED
:1033800005D0A81DC0B200210623FDF7F5FA236879
:1033900004210B4205D0A81DC0B202220623FDF76E
:1033A000EBFA236808210B4205D0681CC0B2072243
:1033B0000223FDF7E1FA2368DA0606D5681CC0B2DD
:1033C000042102220623FDF7D7FA23689A0606D5C0
:1033D000681CC0B2002102220623FDF7CDFA236843
:1033E0005A0606D5681CC0B2042107220223FDF745
:1033F000C3FA23681A0607D5281C09300222C0B276
:103400000821131CFDF7B8FA2368DA050BD5EDB2D5
:10341000281C0930C0B20B210A35FDF797FAE8B233
:103420000A21FDF793FA013604340C370B2E00D035
:10343000BAE61B4803210622FDF7BEFA194D1A4EC3
:103440001A4F0024019A2B78D35C6A781A4205D06F
:10345000A3009859395D0922FDF722FB013402359A
:10346000092CEFD1FFF732FA002814D006240321EB
:10347000201C00F0DFF80321C5B2201C00F030F959
:10348000281CC9B2FDF762FA092C01D10B24EEE722
:1034900001340E2CEBDDFDF7D9F905B0F0BDC046C7
:1034A000133800006C00001074010010A40000101C
:1034B00070B5041CFFF76CFD201CFFF76DFE0A4B76
:1034C0001B78002B0ED0201CFFF7FAFD074CC823F9
:1034D0005B00074EE518211C301C5034FEF74EFAF5
:1034E000AC42F8D1002070BD7903001060130010C9
:1034F000E437000008B5002805D0FDF77CF907483F
:10350000FFF7D6FF08E0FDF77EF9054B1B78002B8F
:1035100002D00448FEF732FA08BDC046A6050010E6
:1035200079030010F97A000000B5FEE700B5FEE768
:1035300008B50A4B0A4A0B4903E0107801321870AB
:1035400001338B42F9D3084B0849002201E01A707D
:1035500001338B42FBD3FCF71FFFFEE70000001096
:10356000507B000098010010980100101C150010FD
:1035700002B4714649084900095C49008E4402BC06
:103580007047C04603B47146490840004900095AD3
:1035900049008E4403BC7047002934D00123002227
:1035A00010B488422CD301242407A14204D28142C2
:1035B00002D209011B01F8E7E400A14204D28142D2
:1035C00002D249005B00F8E7884201D3401A1A434F
:1035D0004C08A04202D3001B5C0822438C08A04286
:1035E00002D3001B9C082243CC08A04202D3001B3C
:1035F000DC082243002803D01B0901D00909E3E7B6
:10360000101C10BC7047002801D00020C04307B434
:10361000024802A14018029003BDC046D900000034
:103620000029F0D003B5FFF7B9FF0EBC4243891A59
:103630001847C046002941D010B4041C4C40A44691
:1036400001230022002900D54942002800D540422C
:1036500088422CD301242407A14204D2814202D201
:1036600009011B01F8E7E400A14204D2814202D221
:1036700049005B00F8E7884201D3401A1A434C081E
:10368000A04202D3001B5C0822438C08A04202D354
:10369000001B9C082243CC08A04202D3001BDC087C
:1036A0002243002803D01B0901D00909E3E7101CBD
:1036B0006446002C00D5404210BC7047002806D05C
:1036C00003DB0020C043400801E08020000607B46F
:1036D000024802A14018029003BDC0461900000034
:1036E0000029EBD003B5FFF7A7FF0EBC4243891AB0
:1036F0001847C0467047C04600B5002905D00023D2
:103700000139037001300029FAD100BDF8B5041C5D
:10371000A30719D1231C04CB0F4D104E5019904311
:10372000021C201C32420FD1181C0B4F04CBD519A0
:103730009543354208D1181C074F04CBD519954342
:103740003542F1D000E001300378002BFBD1FEF7C9
:1037500076F9201CF8BDC046FFFEFEFE808080800A
:1037600053455249414C20434F4E534F4C45002541
:10377000732072656164790D0A00444D313543430D
:10378000000D0A4279652E2E2E0D0A002573202584
:1037900073202573004D454D383000563400257890
:1037A000000D0A253032782020000D0A413A200011
:1037B000202025633A20000D0A4D3A2000202047A2
:1037C0003A20253032780D0A0057616974696E67B6
:1037D00020666F7220646174612E2E2E0D0A0052D5
:1037E0006561642025730D0A004F4B004641494C2A
:1037F000454400656E61626C656400646973616272
:103800006C6564004C4344206465627567202573D1
:103810000D0A0003030000000303005C0003030C17
:10382000000C03037C287C03037C447C03032410EA
:103830004803032854080303000C00030338440022
:103840000303443800030320100803031038100357
:103850000380400003031010100303004000030323
:1038600020100803033844380303007C000303647A
:103870005448030344542803031C107C03034C5492
:10388000240303385420030304740C03032854282E
:10389000030308543803030050000303805000035F
:1038A0000310284403032828280303442810030393
:1038B0000454080303384C5C030378147803037C36
:1038C0005428030338444403037C443803037C54E2
:1038D0004403037C1404030338443403037C107C46
:1038E0000303007C00030320403C03037C106C03B3
:1038F000037C404003037C087C03037C047C0303BB
:103900007C447C03037C1408030338447803037C61
:10391000146803034854240303047C0403037C4019
:103920007C03033C403C03037C207C03036C106C51
:1039300003031C601C030364544C03037C44000316
:10394000030810200303447C000303080408030356
:1039500080808003030408000007080400000000C2
:10396000BF01BF010905000007000700070007139A
:103970000A00002000E400FC003F00E700FC003FDC
:10398000002700040F0800000C011E01FF03FF03C5
:103990002201E201C2190D00000E001F0011019169
:1039A00001FF007E00FC00FE0113011101F001E0A7
:1039B000140A0000EE00FF0111011101BF01EE0029
:1039C000E00130011001050300000F000F0A05009F
:1039D00000F800FE03070701040B060000000001C9
:1039E000040707FE03F80F08000000000A000E009D
:1039F0001F001F000E000A11090000100010001027
:103A000000FE00FE0010001000100804000000047A
:103A1000800780030D070000100010001000100048
:103A2000100010080400000000800180010D070054
:103A30000C000FC003F0003C000F00030F08000053
:103A4000FE00FF01010101010101FF01FE1008005C
:103A500000000002010201FF01FF0100010001104E
:103A60000800008601C7016101210131011F010E1B
:103A7000010F08000082008301110111011101FFF3
:103A800001EE11090000300038002C002600FF0173
:103A9000FF012000200F08000080009F011F01117E
:103AA000011101F101E10F080000FC00FE010B0112
:103AB00009010901F901F00F08000001000100C12E
:103AC00001F1013D000F00030F080000EE00FF01AF
:103AD000110111011101FF01EE0F0800001E003F4E
:103AE0000121012101A101FF007E08040000000066
:103AF0008C018C010804000000048C078C0312095F
:103B00000000200070005000D80088008C010401E3
:103B1000040111090000480048004800480048001E
:103B2000480048004811090000040104018C018884
:103B300000D80050007000200D07000002000300B4
:103B4000B101B9010F0006190D0000F800FC0106D3
:103B500003FB06FD0505050505FD05FF050601FC42
:103B600001F8120900008001F0017C004F004F00B5
:103B70007C00F00180010F080000FF01FF0111012E
:103B800011011F01FE01E0110900007C00FE00830D
:103B90000101010101010183018211090000FF01FE
:103BA000FF010101010101018301FE007C100800F9
:103BB00000FF01FF01110111011101110111010F9C
:103BC000080000FF01FF01110011001100110001A8
:103BD000120900007C00FE00830101012101210186
:103BE000E301E20112090000FF01FF0110001000D3
:103BF00010001000FF01FF010A0500000101FF0194
:103C0000FF0101010B060001000101010101FF019B
:103C1000FF10080000FF01FF0138006C00C60083A0
:103C200001010110080000FF01FF01000100010077
:103C30000100010001160B0000FF01FF010F003C15
:103C400000F000F0003C000F00FF01FF011209002E
:103C500000FF01FF010F001C007000E001FF01FFE9
:103C600001130A00007C00FE008301010101010133
:103C7000018301FE007C0F080000FF01FF0121000D
:103C8000210021003F001E140A00007C00FE00837A
:103C9000010101010101038307FE047C04120900F4
:103CA00000FF01FF01210021007100DF008E0100F3
:103CB00001110900008E009F011101110111011174
:103CC00001F301E211090000010001000100FF0100
:103CD000FF010100010001110900007F00FF0080C9
:103CE00001000100018001FF007F110900000700B1
:103CF0001F007800E001E00178001F0007190D00A7
:103D0000000F007F00F001E0017C001F001F007C1D
:103D100000E001F0017F000F120900008301C701DC
:103D20006C00380038006C00C701830111090000E5
:103D3000010007001E00F801F8011E000700011233
:103D40000900008101C1016101310119010D010763
:103D500001030100070008000A01001811101338C0
:103D600031303378717073C8C1C0C3888180838457
:103D7000848782C5C4C7C2757477723534373215EB
:103D800014171202070208020100030109030402CA
:103D9000040205030500064669726D7761726520AD
:103DA00025735F25735F56340D0A00436F6D6D6197
:103DB0006E64202020204465736372697074696F9B
:103DC0006E257300252D3130732025732573000D6A
:103DD0000A5479706520273C636F6D6D616E642DA8
:103DE0006E616D653E203F2720666F7220706172A4
:103DF000616D730D0A00557074696D6520257573CA
:103E00000D0A003F0025730D0A0D0A00564F594157
:103E1000474552203E3E200025630048656C7000F7
:103E20004E6F20706172616D73004B657920707206
:103E3000657373003C6B6579313E203C6B6579326C
:103E40003E202E2E2E0044756D70206D656D6F72B4
:103E500079006C004C6F6164206D656D6F72790044
:103E60007400546F67676C6520646973706C617966
:103E7000206F757470757420746F20636F6E736F2C
:103E80006C650000008001500080025000800350EB
:103E9000FC3F0150FC3F0250FC3F03502573547916
:103EA000706520273F2720666F722061206C697340
:103EB00074206F6620617661696C61626C65206355
:103EC0006F6D6D616E6473257300A106C105557534
:103ED00020C5F0A0B08E453502DC312B1017134FF2
:103EE0009CC300E302044A116A596686E294CF102B
:103EF0000CB0065A0482F00020C24A00DE1DE22EF9
:103F00000277590555B5414D4999918A08729584B2
:103F1000035555654753256A41C99A107604310106
:103F2000C0C0B40F44F080544599599D8821323562
:103F3000880B04820310D5DE4012150066C43330AE
:103F400009401904508050508E5024A46A0021204A
:103F50008A400156552521218490D1646346A216DA
:103F6000D8A410602254423044744A881115146950
:103F70005520B8072678100846002C06885C0909E9
:103F80000200000000000000000000100300808C10
:103F90000831212310C14110130011D025D8C74486
:103FA00031A188B7A061BB987363501021FB4026F4
:103FB00011852048529110885801008488023031C0
:103FC000006288CE3C0044511444898988B8BBAA59
:103FD000AB2B1221003233232213757700C0CC445F
:103FE0004566B9BB45B4BBB888894030885DF833B5
:103FF00033D1467844EC0010519D2ED1552522A294
:1040000000019099D9DDFDFFFF03C1088C302148E4
:10401000844C0001D34C4802D8940CBEF240B0C48A
:104020003C0C8A37120E59DF049DF14D100EE4232B
:104030003F001232135011FB0C088CC0400101AC40
:104040001336C804599D531659DFDF1C76B3CCB81C
:10405000D30E8803018410D071A1885335D2ED505E
:10406000F04404C900D160F3E24E0C4A2703250155
:10407000130973390CD8FDDD335D7C13163923CA5F
:104080002710102520560C8C443B5114318413D03A
:104090000E6BBCC784EC3A120729C400C43328173E
:1040A000188010C9442D63E022084548D1FC0D3F1B
:1040B000C8FF480F0C0C0C0044328C7D1001A12469
:1040C000170F481DF2760924B70FAA0A2010AA0A72
:1040D000109340230011A4884C70CC12A31C0572CD
:1040E000801DFEC45CDC4518D4F9001B13855B28D9
:1040F000843F0F0CC62C41CC473C414C473FA66D3A
:104100004B1B102F49515A1C17731041C700B06147
:104110003E1D5A1444FC813136463D48C00C513096
:104120001180C41C08C22183CC0C313311D15060E2
:10413000B13E4721840C4C14F1CC0F03CD700467C1
:104140003192BBCB3300282333F100B3C6000448BF
:10415000C010222B1F6A33EDC1A8C11803345004CC
:104160008282A2A00710462466369F04351789A0D4
:10417000D42C3EFD7E008F8D7D3113CA30623C4CC5
:1041800084E020B654F184F640282EED3543150026
:1041900044E2C86114F111D507D04F4C37200730E5
:1041A000C9F1BC348BD29E615020AC547685D102CB
:1041B0004BD80D4D043348814C11CC481014C15CD0
:1041C000684C43A141D98C7B0F0091301A074338CA
:1041D000404C4F0800C03040A802C04444C15404C1
:1041E0000133F9471138453188EC04121000000002
:1041F000310424044C9381C00C00003002100243AF
:10420000147140084C0C02C0880C7037A8090020BB
:1042100031032C0012302348088423210386101A0E
:10422000E28A47C8A800E160A06E08205020C8407C
:104230002420C84000C68C008DC08884204A4C08C9
:104240002182000220444004C4930220A008325876
:10425000E54110BF741D48F4841C9C0320A584A074
:10426000FC3D3008C0D280C4F4432C82A812B111A6
:104270000641F4A1636C72890820134212B0014018
:10428000088042408AE4937F24CD03178282C31CB6
:10429000F2FB000C140C0460631800311048140782
:1042A0001002044A8A01D336D8BD138C080182A0BB
:1042B00028CB00100B2050428155CF838DDDFB337E
:1042C000000B0000804064F9BE26C107034CD80DE6
:1042D00001825550D14FFC0452F1074515407C0036
:1042E00011014442BD43CB4008820C08820C0832C5
:1042F000500CE00021002120412204C4F958D8C408
:10430000D304118D4D464CD30E91AA0CA004AE38A7
:10431000BF87B807FF378E8B2C71C7D9B80F1447EA
:10432000082E8A0720FF424FED4700360104E38C38
:104330004310F4760BA2788CB349480012626017E0
:104340003B020018B248B84354085400E25E199486
:104350002C719B0103648816638295D544422135F4
:1043600003A4041D6014072029D0D90A803020E25C
:10437000FE42A518880009680A0045A22461C029E8
:1043800035728C5F2016640F31045DEBEE95F20CF4
:104390003FA73510E24C431041C8C3BC34D3302989
:1043A000F140E6F823124EC4713D379F2BF77A1384
:1043B000AD1BC4103FA85606A2FCA090D2C61FEFAA
:1043C0004F450200550031088002228403484432E0
:1043D00030A38BC2A24B88C0000EB0359381408EB3
:1043E0004C041601C18D6098418E04862806D0C405
:1043F0004C040A312302028130117200098612B383
:10440000C774C403309530C021F0123031C12F5E23
:10441000002241B1105402C5805412317280EC9CCC
:104420008328CD0432D2C8C858CA4852858C6085CA
:104430008C24858C60C55032125429236225234870
:104440009532B25621C830A2C4C452100544515509
:1044500011114A5554554985085E12445544451476
:104460009415554554557454D1552195CBC4051018
:10447000C509C13009022042204CE18E8EAB4F208D
:1044800010B9E4C6FFFF4D1763CA00F2299D30142E
:104490008F5111A036120412D0E54948507AE477C2
:1044A000086109EA440D2060A03E80820A220514BA
:1044B0003C445F0414420445421253806541404C21
:1044C0004C0462C82120C4A841F2061A1510201518
:1044D000051455104CCC540140A02C2E400C005912
:1044E000260413310E101333527446300A0401317E
:1044F000120C44440082C08CE0133130003232266A
:104500008C4081000281840231003144000144006A
:10451000000011D388C80018480404008824C0C4CF
:104520000484342EE2A2C82227C004310A301320AA
:104530008404083044D0CC144D044CC8C484444294
:10454000C320F020201004451005110F00229C0C00
:1045500001004C9301C3C0091688C01012323010FC
:104560001220444C1854804505985008E300850CEF
:1045700012822404000481080D2010201088448435
:104580000048301186844012001133338D60800260
:104590000B291180213111500404CC002413D000C8
:1045A0003333A12CA1921A0D05D040390903F284AE
:1045B000901C4D22820DCC30D0941C068AC82C6BE6
:1045C000C3F7C01CA3F079B0820010C848E8888007
:1045D000C212108035C40810115D0205A423804466
:1045E000804091C23BE3400D02208010048E0820E1
:1045F000F33C0F1104897BC35C0031001020507024
:1046000020E8104CA3024E86D6101D384C830106BC
:1046100075CBA63C309EA218B0C9F318C8A030A430
:1046200020133138D3915890043D8A67802003E1EC
:10463000345D0C1434104810B4807319D49130D305
:104640001441180B10871C3210618C3912104C0366
:104650002110142412417DC86C18C6D6DD10121A20
:1046600037305E22F15C08353D62563C08A248387E
:104670000788D825C619CF15B01D152386E08620DA
:1046800031473104D120903F00008A0B4A50B28854
:104690000150C74462197210C0D8239EC4332C6DD8
:1046A0000F2A584C3C330411CB87A925A184D5147B
:1046B000303E12469852837AAD1C076845A062824C
:1046C000C0303838180130070C00DC043D55320F7B
:1046D00093A104D69716020EC88C848012238BB245
:1046E00082B0AC47420C8DC02410C6334605214928
:1046F0004812928484C963904936489949236011CD
:10470000B684C260B904650F00216433360182E1CA
:10471000144F114098B3DD4BD66A4110C33F1C843F
:104720005C1C43711CC771F12161EFA11D0F3BC0DF
:10473000323C3F31CCF21CFF073B0A9CE010780969
:10474000CE3B82CE7F0412892028D6230D3418C395
:104750004C2033033C4C38474C118470C70B000489
:10476000111151440EF0088C2050FC1189F1445471
:10477000344D4D2C0131F4D33490D0E984818150F3
:10478000F30F024020A3C81F42E48030F3343939CC
:104790001981B3DC0C0183C840D3E424E132C8FCA6
:1047A0004B4C39F18001600981028A0D13010A28FE
:1047B00076F8A000FBF4BF6183BF10106288E3416C
:1047C0000317AE4610DAF33DC7C4400400A14CCC39
:1047D000494851C1120104040F218402224A48149D
:1047E00035104000E30048CCA8C8E844084440A481
:1047F000043A20110312C47808442408002111004F
:104800000061125112481810200112A44540009274
:10481000B24C0C100E1081000010211011A3442185
:1048200060100B2A23B22BA2400A502800110884E2
:10483000028440940C408C00231630023112308ADE
:10484000040E318A440C00A07AA30E4E1C11418440
:104850004430140E53DD124FC411C3C44F1027450A
:10486000C7F43C06AB33314371B8C3A03A9FC1646F
:1048700010B31BE318443162A82D974CC81148C4EB
:1048800008034062CC021D1A682023C655618B8A3A
:1048900038CD92820CC620D4C43436B2C40535401B
:1048A0000912880A3FE23BF5124C4577C794E9F6B6
:1048B0000C458084A210C85096FB202185C5EA2FA4
:1048C0001280003B70740914900095820604102039
:1048D00044003000407028140350084144984103BC
:1048E0004020020C01B123CF49330C0311F14704DE
:1048F0000D180319D260931803B1AA03408D070461
:1049000073047DE300D0041110D316911431D1103B
:10491000C30010640460000CC0C0000444BE6450B6
:10492000D086983B314414330001C83001813311E3
:104930008D99049D91D38C4DE444A42C24312251B3
:1049400011E51F00310D441E533D144021600862E3
:10495000583644144913219C2C11B04C22238064F6
:104960009F0CA1D2594C4CB9409574540C22183B61
:104970001085DB208A0F14430418308CE8408091A6
:1049800001490183040C1C43884C11FBA118B03968
:10499000099D363F7240030E31404B1253E0904464
:1049A0003E4D044140D065B218F4134352D5E38F15
:1049B0008499DB14A6044C282B638C28211C1ECC64
:1049C000C523885C7AD5A1C1CEC8013CA0000C04E7
:1049D0003F3CD74040C4144A00F0448004031A8A84
:1049E000C348F101D5044404A2A4306B4564884453
:1049F00011C10061C0E10013C117860230122747C0
:104A000010A144CD298113A3024433340A84020047
:104A1000012C6C50A1C7D74344C82412A082C3C53F
:104A2000F1FC7F32FCC4E8F24444300001CC4C007D
:104A3000109052531C9D004390614CFC81311881B1
:104A4000250C84E0C4AB03315900008110440007F9
:104A5000C4344B847D158E048034112211090882E0
:104A600010224E00130C828807190E3407583D108F
:104A7000110B037F100B651405F30F4C4E04184205
:104A80000A5D0FF2AAD88B930821F5E28698C9D463
:104A90004074BAB274A4364D72601D19494FCFF4F8
:104AA00087F04C4C44401841045828180441883A77
:104AB000DFBDBD7B1FFF3112868E0A023EC0C821BA
:104AC00055882088EA1C3B000000CF4E7038EE0F5E
:104AD00041A0210C6E0484A50200BCFB3279401376
:104AE000CE35244E203C063018E06500666071AC7F
:104AF000E0A94E4E5C2650E00080B4EFDF7823073B
:104B00008BEBC241A06500668784210C3D4C0404F8
:104B1000448465003075666330176673301266CD65
:104B20005A3014665B2666CF883D4CB95C8CEF1C0E
:104B3000E0207314FB8100C360003B02E07724D0C7
:104B400043ECC9DC101EF81EE83357CA06751B4536
:104B50000E12B84E20305ABC70E0E0D59C619C33F8
:104B60000ED9A0D99C01401B04044419A410A884A8
:104B700004446EE59C6E0CE5370CDD37048CA923EC
:104B800049BCA9A8854E480940134429E176FCFD9B
:104B900000EDAD1C621C629CC906CC4714B7D4B7AB
:104BA000543794B90ACC7FB67F6666CCEB666666EE
:104BB00099A8B61CCB666694C7CC9399A8B6B69C48
:104BC000A2E202DCC83366CC47D433CC231CD08DA0
:104BD0000ACC3F142BCC5D0B5C66666666CC4794B2
:104BE0003714654F81A866666666666666666666A1
:104BF000CC9754B7540B56E33010C6B3CC37E3CC44
:104C0000DB666699A8B6B69CC833CC8F947B99A80E
:104C10001CC8BB66E6438C079467545714479443FB
:104C2000CC2F2BDC2B5C444C47E616B6DCD4EB8651
:104C3000A6445459229D2EE01CEAA04884854E6665
:104C4000666666F8FC941FD43754279417541F14D3
:104C50000F1433F6D3D016D3F667CC63E616767608
:104C60008648845C53CCB35C23CC3F1C85A8C471BC
:104C7000061CE399A82399A8669C6666668BCCA758
:104C800094AF99A8C8E3CC4FF846E8941D1F911E35
:104C900099A89C83CC659F945F8C31A7542B71ACF1
:104CA0001D529C710ACC3F99A8B65C236699A85CFA
:104CB0007D0699A8B61CC87506CC410794CF99A863
:104CC00066665CF502CC450794319F5BCC69232B6B
:104CD00014A7CCFF5403CCF3065CC906142BCC6795
:104CE000610ACC4F73148BCC17666681A8DC1366FF
:104CF0006666666666666666CC3F941F5C231C1318
:104D00009C85A87D06141BCCAFCCA7947723945721
:104D100014E714AFD48FCCA59F94B3CCA31C9016EA
:104D20005394B714BF1433661CC47906141BCCA368
:104D3000541FD497CC950A6B66661C89066699A8A1
:104D40001C7506663366CC271C621CC106F8FCF68F
:104D500063D0164B3030066666CC1766305046C4BA
:104D6000C3666666666681A89C91061C1010E646BE
:104D700046B63C02C49906CC6F9449076699A81CB4
:104D80008D06CC519F94859F99A8C8A3CC27C89421
:104D900093DC73CC5714431C62629CC4C82B9CC424
:104DA00044C4854E133373C38382C27232121030EF
:104DB00070C08087C7773717113171C18184C4747F
:104DC0003414183878C88884C57535157140D540B5
:104DD000C14CF5A871400E882B7140B0AECDAC85AA
:104DE00038C9ACBE5541F1404938A188C1AC8D38B5
:104DF0006140DD40C14CB14C8C6055A4AE2871407F
:104E0000C5404938A14C7940D540C14C65448DAC72
:104E100038E03051A6A64E70F866A030049C583099
:104E20008006301BA5A86DA4DC10105090D4EB6850
:104E3000C4C44E9C90A8A0706E1C5090D0654EDCEF
:104E400050D4F34CA0EEE04E70F83CE6BCE8E580B0
:104E5000B9A028E6F62B9A26E3FA46BEBA0E666893
:104E60009C0AED4CB9A0A8F14CFA1F4E224C17BE7B
:104E7000AE38FD40280E78BE1EFD40AEF83C5670A0
:104E8000AEF04E70B80E384C4FEB0E330EAE1B3DED
:104E9000ACB940BEA74EEEA70C834C7701BC0E48C0
:104EA00021BE0E1B0EAEB940FEF59C81024EEED720
:104EB0000CD34CC743000000000000BC88E4E8D8D5
:104EC000787CA8FCF844404CF474DC48A5363D32AC
:104ED000B896913387349D26DCA3DBA4DDA5B3917E
:104EE000B9928993DD149115A0FB1A4833366331CA
:104EF0004A169533B5348C26D5A3D6A4D7A5A3914D
:104F0000B792BB93B5943B95D8FB8300E201EA02CC
:104F10002003BBD3BCD4BAD59821713177308940F6
:104F20003E30743110320649BEFFC300E601EB0289
:104F30002A031ED3EED4FFD5ED07EF08F1098A400E
:104F40003244002006108549B04C7719AC580C2B20
:104F500021BC4EF04E7098E05819A4E28BBB9DC066
:104F60009AB085A04D908649D8E00048493635353D
:104F700033442B251B3408200B49002100520062CA
:104F800047754274323053435843401638268F23B6
:104F9000B623E804F405FF060C070E0810094716AF
:104FA00069160B100A2066040E050D066C4077305A
:104FB0007B2080106B4075307A207E10CCD8DAC20E
:104FC000C0E3CBDCDBC3E40CD18059A40C21BD21B0
:104FD0008C7D8AF510813CF0CD8CA18839880C79C4
:104FE0008F654421AC1532F51061406588704D40E5
:104FF000653C630EF3818CE32E0E7AFE4B48CC3376
:10500000CC23C488445CA606E669174687CECE2327
:105010005C62EE4F4C0761A00EA6AEBB4CA13F0DEB
:105020003C818C46936ECE5C5A5E26E6433ED45459
:10503000D3EEE116D84E3ECE6BAED8221ED8AEAE21
:10504000BEEB1E2EAE8ECE93D83ED86EEED454B3A9
:10505000EED93C6ED8469C7D14EE132E62F38E4240
:10506000FAF3DCA34CBB794079407940A1888540B4
:105070004938D14C213C1EA606E655166D16DC6655
:1050800054EB5EFD38CC3BBEBE11A00D408C2B1105
:10509000A00D404C8766660011A08D3C8C3F4E5C95
:1050A00066508D384C1BBE1EE0EE4E6E5E546F9403
:1050B000E7D41F5447145F9CD09CE0DC9090109084
:1050C0005090105030165CE09094F36B1CF9149CD7
:1050D000505C109CE05CF9149C50DCE05CF9145CC2
:1050E000E01CF9141CE0C8481B0EBAFE43884C1B98
:1050F000CC13485EEECE5AF6137AFA4CF78C2BAEF0
:105100000ECECE4E5C1050EE6AFA2F6A1B2A8EEE3F
:1051100058EEEEEECEEEFA9F8EFB2EEE66DB4EEEF6
:1051200098EE4C1B8ECEEE8E5B2EEE98EE4C0BE680
:10513000F7EEEBCC5FC84C37487361A0A3444BC477
:105140004CAB8C1B841388036E8E00818C3B26F63F
:10515000278EB32E6600FD384C5F98EE6600853CC6
:1051600011A09538D8AE0E263B6EEE3BD454AF2638
:10517000E36E4E7D14EE133E8EF32ED4CEEE54A38A
:10518000D88E8E4E5C50D89C90905B8A8ABEEB1E67
:10519000D8AE4E2ED88E1E62ABAEFAAEFA737E66D5
:1051A0001E8E9B98CCB7CCA30D3C8B5ED8AE98AE30
:1051B000CC1FCC1F866EDA73D8C13C4C4B7940FDB6
:1051C00084CC3F0D3C4CA0BEE0B058468C213C8CBA
:1051D0000D3DA1882938CCA1898CF1CDA188653CF1
:1051E0004CA0BEF1CF4E5C7A360E8E4CA0730801F7
:1051F000A48C33F59C15CCBBE6E784EEBB9CE22384
:10520000C1CC9BE1A01EBED05CA20645543D4CDD46
:1052100036B1A801A408059C8C1F888415CC9B2856
:1052200005A84E7038B1A85E5AF643880656BC668B
:10523000B6CEEE0DA406781CEA4B6A4F1C908C1774
:105240003616C12EF99C8CF99D5658F59C06567061
:10525000381E1AEEB61C23DCDC7CB6E316EE7CCAE4
:10526000CA8C43D497DCDC7CCACA6E0EEE0E7C1C62
:105270008C1B1C7CEEC3C2D4C2AEFC1CEAEECE7CFE
:10528000AE1C5BA6AE0E70387C8C137CEAF0986680
:105290009F91CC84491E8C6BED80B9A060E6235CA5
:1052A000154E7C0630089C6217484E3613EEA2F36A
:1052B00069A4B8AEE0CA0A0ACAEAEA4A8C330E0602
:1052C0000E46E04ACAEAEFE00000505D707D909D16
:1052D0003D3E1E2EC8019248F50E515E717E919E94
:1052E0004D4E9D9E79CC8C4BB8E633A646A8A5A81A
:1052F0008102ADAEB1A801A4E1A01EBED05CA2E6C1
:105300006365CC8C236D202B886D2084068CE10393
:1053100045543D4CE065CC0C15A00ED8AE8CBD03B9
:105320008C551FB1A8608444064E701C56792330FA
:10533000FA621F069F30A806BF62CB30B0C6161CAB
:10534000108ECAEABC30063A308C152F0C33D88C3C
:10535000798FD84E3096BC704E1C1006BC70CE6251
:10536000E21B380EB0A0E08CDD2FE6E69D3A00622D
:105370001F024B3030063B8C052A30B0CB30500634
:105380002B48C38816300A9C022730B24B30700677
:1053900033764830AC1B1C62DB4E1CD01006BC3090
:1053A00096069C021388566376BBC9B830301C0A37
:1053B0003F16E202138430C203764B5C6262C8433C
:1053C000765B1CA2304006174830D85B762330DA73
:1053D0002B763B30E24899B85A5E861686064646DA
:1053E0001C10068C912BBC30064E1C1046309BBC0A
:1053F000704EA6BC6E70B04CA04425BA4E1C100274
:10540000D09006BC305AA03DACBC705394F981F0EA
:1054100023F910AECCA07039B8CCF59C0B21B8AEF6
:10542000619E21B859A478EE5670EE0924619C8BD8
:105430000924AE6D02C89940CCD76544F0B0ABC822
:10544000AEB940ABC855388BAEC8613C63B0B1B89B
:105450004613A64E300979A83B9C4EA22805A84EBB
:1054600070388C539C222233998C548DD758A0B01D
:10547000FA63EE59A4FA3BB1B86EAEB1B8B9A8EB75
:105480008C53300E9C629F998C540779AC8E6524A6
:10549000EE3C066524F5A8EEE0F91049A4FC1C0AD0
:1054A0003C6ACA1681CC605E7CFAA0265CE260FC95
:1054B00046E0311C704C2BCDA80813A88102311C8A
:1054C000AE00B04CBB0405A8A3311C4C230C7723C1
:1054D000B03CE6F59C3B10235013908C2FA25895BE
:1054E0000206ED80A61C58A6B9A0FE4FE61B5C5034
:1054F000DC985C5B0E4EDC605090461F1A171ACE8B
:105500001A7B19A4BC9CA27CA863F9104E9CA23CF7
:105510000B4E9CA20E1CD0BC305A1CD0BC70B03DAF
:10552000ACAE7E4484C4FE1F88C83EAE7EFE1F48DB
:10553000C83EE089284C2BA66DAC7B58A6D5C00E82
:105540003C3370D8F0D826AAD3B0E01CA28103A2C5
:1055500013C88CAB998C949FB9A00EFEDFE6AB4EBE
:10556000DC909050A646171AC12E605C021B76CEC6
:10557000CEFA027C9C02A388465E7C464BFCA64683
:105580002BFCA64627069D2E1C026DA001A4844478
:10559000CC0D2F6E0C770C67089DCCC8CCB123497D
:1055A0004C2922B85CE22F9CE2ADBE9C154E26BC75
:1055B00030D61BBEBE0630501C0A4F30304A7C1C11
:1055C000D0D05BAA1C109016E217625C7C66EBD808
:1055D00084D806101CAA027390BC1C10B61B901332
:1055E000D09090612E0AFC5A7A7C5CE227D05C1342
:1055F0009CB6AF10B67FB67FE6E6B62B101C903B8C
:105600005056DB1B9013D0FB1CD0D0E61630A00602
:10561000CFC6E676541B5C23FC9CD08C1F501390A5
:10562000EAAA1C224BD01CAAE0E65CD0A362A6BE6C
:10563000B33A46F12E84A04E30493606F3600DA4ED
:10564000E6CBEEAE0EBCFA4EDC901AEE1A7E3F1A96
:10565000FAFA1AFAB31ABA30FFDC90FE061C707E12
:105660009E387C361FBA573CBED3A62A77A6067B47
:105670007E9EBEBCB6CA6A3736275C194E7601A438
:10568000A6AD9C059C0679A431A48C092B0C470C73
:1056900037B85E5AA84EA6E81936981BB07C869C8F
:1056A00006301070603008626F787C0C2B06300575
:1056B000463C30803362783C62F3661C56E66036C6
:1056C000E05CD0D0F92E00000000300A0660C92648
:1056D000150E7EFE8DD77C0EE12A39CC663006068B
:1056E000A5A84E705B3009512C067CA5A83010701F
:1056F0004E2868A893F980CDA8619C0821BC934EE0
:105700007019A410A8489502F980CDA80821BC0EF4
:10571000B09926F910A079A4FA5C5050D010D0505E
:1057200090909050237AFA7ADC133A62F354BB6972
:10573000483A38BA28BA4E66FD3963F910A079A400
:10574000ABF980F6332627DAFAE7BA79A4BAF0B0D3
:105750006B45BE8889284CF1CB095699AC99AC9918
:10576000ACE3F910C1CCBBF91011A0EE3A467BF9BD
:10577000100C4319BC5821BC98F06DA4F86D02E5DB
:10578000ACE35EE0C84801504C378C3301A0CB8CB1
:10579000605E054479404CB3E14CE140CC6735385C
:1057A000AE58B01E98BE1EAEE0A18879400D3C6D8B
:1057B00040CC1F353AE14C4B01A0F5407940B00197
:1057C000A01138993C6D40B54A01508C600E5CA226
:1057D0004A2F4E7A365B0EFD401E7940B05E01A026
:1057E000F940553CB548513201508C60CD38794074
:1057F00031887940553CB05E0540B548CB19ACF1D5
:105800000201A4E677B1A80DA4440C9F0C9779CCB3
:1058100084B3CC2B81008C2B6E65CC6E6522048406
:10582000C1CCE637EED704BD02F637B19601A40C21
:10583000570CCF0884E6B123C51EF59C844B45BCAC
:10584000E04554461C1066FB0C15A19502355288A4
:105850007DACD180280E4C23C1AC1BC9ACE9CC2D4A
:105860004059A438CD384C23BDAC1BC5ACE9CC3570
:105870004059A44C1F48F30EB08538E9CCB9AC357B
:10588000400E62E9CCCDAC2D40D59CF1027DAC310F
:10589000ACC1ACAEFA271C154E7D3CEDA831ACC9AD
:1058A000ACAE7D3C6D027DAC44CDAC2EFAAE8540F5
:1058B00079404C272D401BC540B14CDD40C14CA167
:1058C0004C4C27284823EDA838DB7DACD9A03D0EF1
:1058D0007DAC090C837DACC9ACEEC1ACF5A8EE2B58
:1058E0000CC748B38CDF4806B07DA01C625BEADCC5
:1058F000E38C1F44A30CAF8BA214FFD4274C177E5C
:10590000D4D48EAAEE3CDCCABCAEEE5C1EA05AAF6C
:105910000EAE6E738C1B0CC7FAA1028928CCD1CBBA
:10592000BE44F0B34267A6FAE326935CEA8EB0A0C9
:105930009CC54086061CD62B8A838A06AEFCAE2602
:105940001C5E2FA6EE8ADBA66E6544546D029B9CFE
:10595000A2A2A2D384488CD789A0442E5C22029CA8
:10596000D84670F8AAA6E8A6AAD86A085A0F046A08
:10597000F3FA13EEDCD0EE3EB30CA72E1B0E6B1920
:105980004A0546F54A0EA14884B08D38514EFD4077
:10599000230EBEC74D40CB4E5C665093DD408BDD81
:1059A000805D28CC7DC32BD18066662E7A58463E1A
:1059B0005ED8065E139E0ED8DCDC8E132E62F35486
:1059C000CB98AE58FE1B66CEAE5C4AD7EEAE5C0EF0
:1059D000E66B3A5BC62622DE6EFA604E1EE0C6C358
:1059E0004D40A06E4B423766EAE30E11A0EEB08D3B
:1059F00038A500C30EA500853811A093881D448CDE
:105A00004B98D44A538928CC9DC72EFAAE4ED84E17
:105A10005C50EEAED8AEBBFABB693CB36140A34D5F
:105A20004063DD805D28CCA1C32E7A58463EFAA1A2
:105A30003ED8465E139ED85EAE6E2E2BD8EE66D84C
:105A40005C4E13228EF32EEED4D4D3AE98093E5D75
:105A5000384502F5484E58A148EE9BD180F54038B4
:105A600066660043C1405BA140432980232EFAAE05
:105A70007E239C154E1E3ECEEE113E6EEEEE0EEED9
:105A80005A0EE62BAEBA0EEEEE4E9C4217AE8E4E7E
:105A90006EDC50CE4B22CEF34EEE94F7D4CAC3C880
:105AA00048A5A07D1AC848C8A5A0B916A5A0751616
:105AB000A5A025168809A642231013503C1EF8FC09
:105AC000D88404D83C601EE895026544F08CA01987
:105AD000A45C84903B2E7A05406544F0FB5C500545
:105AE000403B0E2E7AE32D404E7078A83868CEBE2B
:105AF0001E28F8BA9CEAEAEABAE8AA8A8A8AEBF18E
:105B0000404E70EED8F81A9ABABABA1CEAE6E838EB
:105B1000EE7828B868BA463CFED8EE5CE030049CCB
:105B2000737030051C4BA1881B794030069C70387F
:105B3000EED8F8D4CE14EBFEAED80BC1AC1D38793C
:105B40004031ACBDACDBC9ACAEC1AC21387940CD85
:105B5000ACAEB9AC63C9AC1D387940CDACAEC5AC08
:105B60008538DD404B4D40EB4E231E4EBE5C50E36E
:105B7000DD805D28CC29C393DD805D28CC4DC34BEF
:105B8000BE5761404B0E78AEBE2E7A58463E5ED868
:105B90001CD4763654E3EEEE6BD86EEE4B2687D8E7
:105BA0006E26DFAED80E23D8AE2BD8AED86E9E5E52
:105BB0005B8E1E263BD8FCD86EA66E264B66CEBEEC
:105BC0001ED4D4C34EAE98EE2E767676767600E16D
:105BD0003A2EFAAEA0DCCED86ECEF66026E63B6654
:105BE000EE1ED44ECF66E0A643A13EFEEFF6DF0EDA
:105BF0008E1CEE8A5C4A8F66061B36E04E22CE3E35
:105C0000EEC21BAA260EC223EE2EFBDE338A6E26C0
:105C10002EFB6A626B7E5BEE865A5E2A4EBAE04DC0
:105C2000408D3CFA174EA05CF62B86F61F86E0F6F8
:105C30001F4E334A6A5688D4D4E0BE6E8E588E4EBC
:105C400027980EE026CB5C626EC13E2EFAAE84042D
:105C50005E13081E1A6ECEE673CE5E7FDCD4947996
:105C60004726DBDD48C3A1485C336E66AE333A8E0F
:105C7000F32EEE66539CE22B62E24F225C43AEFAB7
:105C8000AEE26B4E5C6A0E1C500C13A66E0E4C3BC3
:105C900079408540A1888C1BBE1E653E228EF32E66
:105CA0005447EE66D4EE6546EE4C2B4948AE6EDCAA
:105CB000909CFAABDCE22B628E58E3268E7EA346E4
:105CC0003C626E0E0C0D3D3B6E5A5E0E0CC1454C97
:105CD0007941794013AE7EF32E7E98D3588EEEEE46
:105CE000EE0E6ECEEE2798AEE066CB8ED826B13E95
:105CF0000EEE5C90D01090501050105090505010FC
:105D00000B4E54977A103AD4DF5437147F94BF5413
:105D1000E79CD05C6B9050D05010D0501010509039
:105D20005CEEE0D0501050D050101010D0D09C93AA
:105D30001CD0D0101050D03068DC3B5CD0D0D010DC
:105D400010D0505CEB5CD0D030311CB330339C931E
:105D50002EFAAE794084D1805EBB06BAF633A13EFE
:105D6000E6EB66EE5ADFE64FBE1EFEFE1EFE138811
:105D700059A45EB54845022EFAAE48DA7FDD40FAF6
:105D8000F398FEDF2E653E2EFAAE44043E7E871E5B
:105D9000DA6BA606E67B461BA6080E5E5A5C8A6294
:105DA000228E588B5CCE62AE4E314E422766EEE3B9
:105DB000D8C13C8B7940AB44043EAE0E26E6B35EC0
:105DC00057AEC5445C4EA60E6E3B08CB54F7D43E8E
:105DD00026DB7B8E7EF3982EBE3B3E6EEED4949BEC
:105DE000AE8EEAEAEAAE9CD086C6DB5C8EEEDD487B
:105DF000894CFAE3D4BB2E9C822E8E9D480C376EC4
:105E00008E6E2E6E1C894CFA3B8EDBEED38E235E9B
:105E1000EF665E0CF519FD384CA0DD40953898FE14
:105E20001546A6EEDB8E49486E5C232E62F34226B1
:105E3000DCE05E47993ECDAC5846FA31368D3E8562
:105E400040E36140CB66665C4227FAA6E3AEE0849D
:105E5000A00404C4A01BD46694EB606EE6A256179F
:105E6000B6A61C9090901090BCAE1C55544C2903C3
:105E70008C2F0C603D4C4E70606E28F83051A6E8B7
:105E800060001C4610662FC8CCE7934EA8DC9090AB
:105E90001C1010D0109068959EC8CCF73004C8CC68
:105EA00066EBE09CA20242300842DCCC2799A82392
:105EB00099A8B6B6B6B699067940658C29381E9968
:105EC0003CDD428BE5D3C6F50000EE4BF643A63031
:105ED0000786061388D9A2F6FFB9A00EB0CEFE2F12
:105EE0004E8F85464E375C4A2236E0E65B66E643D7
:105EF0004EE0E62366E687F5CC0EB0FD40794079AA
:105F00004029384E5090268D3879404E5C265050AE
:105F10000540D15C1050213C4E26D010D010100509
:105F2000406D40D15C50D0213C4E269050D0505016
:105F3000554061404E5CD08D3861404EBED84E1009
:105F40001010213C4E106605416D40E14C4E66D864
:105F50004E50501050D01050D0D09010D00D406105
:105F600040F1CC0D40A18861404EBE664D41854058
:105F700001484938614011447940F5CC2EFA0E7938
:105F800040DA5BB00540E14CA18885409B614065EB
:105F90003E143F8CD532600CD7DC501C6233542742
:105FA000DC7ED34C3B7E37A2D4442BBE025437B0A8
:105FB000E13A069C4A3704F80AA1025C4A279C028F
:105FC000138A8D3AFE2F1D444EA0A13E15A0D1800C
:105FD000E95059A4E9503DACB01C427FF940FE5F46
:105FE000680EB0288C4FF940FE2B7828B06859A471
:105FF0005CEE1F502B4E50280E78FD4079407855AE
:10600000A46E9B2E7A7940680EB8FD40788C853C52
:106010004938F637434D40653C45025CC44813445B
:10602000846095584E70E0DCD0AE281E5F7E530C25
:106030003B9CE21FD013D05EA83C0E364F85BCD6E9
:106040001B5C903C4EB83C365F85BCD61B9C107CDC
:10605000EEEE4EB83C364F85BCD61B1C103C4EB8FD
:106060007C364F85BCD61B9C10FC4EB8BC36578581
:10607000BCD61390FCEEEE4EAE91580EB87C365F57
:1060800085BCD61B5C90BCEEEE4EB8BC364F85BCD2
:10609000D61B5C90BC4EB83C365F85BCD61B9C10B2
:1060A0003CEEEE4EB87C365F85BCD61B5C107CEEB9
:1060B000EE4EB8FC367F1CE22371BC1B85BCD61BA0
:1060C0009C10FC4EAE7D588C234CFD5BF8FE434E7D
:1060D0003008A8300C3B4E300CA8300868A0381EA1
:1060E0007E077E9F7EC77E677ED35C22AFB87CEE44
:1060F000EE0E7B787C4EB8BCEEEE4E7C1B787C4E70
:106100006E1D5A4DDC0EFC9C02788C234C174EA25F
:1061100097A20FA25FA27FA2F7A25FA27FA2F7A21F
:10612000477B7C4EB87CEEEE4E6EB87CEEEE4EB801
:10613000BC4EC37C4EB8BCEEEE4E6EB83C4E637C9B
:10614000EEEE4E6EB87C4EB8BC4E9CB0FE23109C5A
:10615000427870686E89588C1B4C7FF85A460C1B2D
:106160001C50FEFE3B1C10FE1B1C105EDC8C1350F2
:106170008558F8FC5A46FE235C505E1CCC1B223B23
:10618000A09423E01C50E07158380E8E5C505C6285
:106190004F78BCD88404D8BC68E0208C3F19A45C3C
:1061A000E21330A059A60E7870682B0EB870A88C38
:1061B0002BCCA048E04C60C8CC6088494EA01C1095
:1061C0009C50201378EE68A8863D4C4E5C906EFF84
:1061D000CCEB30DA065ABC3006203C56668F6E6631
:1061E0003028060F4E6E1C50500E55549502664EC8
:1061F000A02660A6E33C315E15A0B028C444415CF3
:10620000D50CAEF0986EBFA01C100626E630187CA8
:10621000BA5CCC2B62622222304613263A7AD786A9
:10622000465F48415CB0CE4E3A30F3A6CC231C907A
:10623000106E5FD50C0E986E2FCC2FC80B4E834E70
:106240007038704E6E68A8CCA08481024E2626CC91
:106250001B26263C134E5CF0154EA0D50CF0F0D852
:10626000D8D8D8D8D8EE6ED50CCE4E5758844E30EC
:1062700007CC2388301A70EE384EAE8C274C7F2E18
:10628000AED8F04E38D8F06E3019667784302A4C8C
:1062900017860698065830187B30E0CC1B30C06655
:1062A000833010662730E0066EEE6656538E008B04
:1062B0006EE0584E7078A84E7038689828E04EBE50
:1062C0002626D84EDC5050905CE01C8540EBBBBAD3
:1062D000974F3F4361407180A18871806D427D8CF2
:1062E00051A91A27C78DAE0E58CE6B79894DB58846
:1062F0004D40B005405D4021BC05426F66743DAC29
:10630000B0E580AE236DA4B87EFE271C154E3EE09E
:10631000CC24525B906140953A918863B58838BE31
:106320002878BE6863B5884D40B08D38F1886140EB
:1063300021BCBE8D391DB8F0E9808D38A18821BC03
:106340008D38614058C98898E078BE681E61401E4B
:106350000D40FAA13E858AFD803BFD80BD88758099
:1063600019BC318C6DA4F8CD8C3180C988493C5D55
:1063700040D54E9188B0FE1348813CB05E05403553
:1063800038993C70FAA0DDACE14C1E4CA05EF0BE2A
:10639000E0D180E1AC70FA2F21BCFA2B01BCFAAF3E
:1063A000198C1E21BCFA2BD188886B7940198CE19D
:1063B000AC703988DD40A188B0318CF18884C14847
:1063C0008588C9884938B1A861882D80619C704D45
:1063D000402D80EBD58884BD88858875808C43D915
:1063E0008461883B9188D98459882D805D40293803
:1063F0002B21BCFA2FED3859028DD899487940D31A
:106400004D40441144A1886142D588984BD5889964
:106410004879408580798E884D8C1B91888D84C900
:10642000882938C9880580F1887D808C4BF0BE377B
:10643000E988FA1BFEC3BEF0EB4D8CF588834D8CCA
:1064400065845B884D8C1B91888D842D8070854080
:106450002938CB4D8C1B91888D8429385D4005806F
:10646000739188C988418CC9883180FA276D1C9B3B
:1064700021BC5E5846213C4E108D38B5485C4E100C
:10648000853C0E21BC1EAE5D404E9005402D806DBA
:1064900040F1CC7140DDACC988318859A478FA1F2D
:1064A000B01E3538F0E09188813C704EE021BC7020
:1064B000ED308C2B318C79407140AE0EDA70048C4B
:1064C000130859880C17847D40A606DA6544845465
:1064D00027D4472E71807940993E1EE04484C4E061
:1064E00048888849886EEE711A0C4321BC5819BC43
:1064F00098F06DA4B0E8E09188619CAE70E08819D6
:106500008C4EAE900EB05EFD40FE33298001487B7C
:106510004D408540A188794049383980B548858803
:10652000A188198C8C1F4888398870C988F18861C6
:1065300084584E70F83CA6BCE83004A34E70F87C3A
:10654000A63CE83005534E70F87CA6BCE8300670D7
:1065500038BE5CEAF0E048884988884D40DA8B5EB6
:10656000231E88C8E14CFA170EFE1348C8ED1661C9
:10657000400611A04C4F4E668C2366501350EEFA25
:10658000653FA0E0C891881E794079408540318000
:10659000993C794085401E79406D40E14CA1888549
:1065A00040418C71801DB8993C4D401E0D40F188D2
:1065B0008540DA213DE140F188E140DD4098FE1B55
:1065C000C988DD407940658CA1883538B94C0D40CB
:1065D000B5480E21BCFA1FB0BE1EAECC13BEFA17D2
:1065E0005EF048C848884484318C6140D54C79407D
:1065F0004EAE698DFE676140DDAC8540213CC5141F
:106600000B6140A188CC2388C413C8F1CCB94CC518
:1066100014DD4098FE53F1CC8C3311A0EE0D406593
:106620003CF0E04E5C900542D8EED8B07EFE439C34
:10663000C23F59A47EFE252298666666064E309EAD
:106640001C90BC70A65A1C90BC305A1C90BC70A008
:1066500021BC58318CB0CD8C79428140E321BC58AB
:10666000B0F0918898BE704B65445821BC98F0B04A
:106670006D02FCFEDEFC06512CE6A675AC31DC6634
:1066800081CCFA3C0681CCBC1A60DECE9C4A6A3AC8
:10669000CC1BD0D0C49CAAE217D09CD0E217D0DC8F
:1066A000D00EE0B05E5CD4A6F3E0CC1FC8E0C4E03E
:1066B0006DA45CB87EFE2F0E7C9C023EE00E2E7A0E
:1066C000E0A7DBD3E8D07100000002A628D18089C2
:1066D000900C1F0C930DA4BCE6852BBCAECC374CA4
:1066E000339C154E8CE7CC2355A8238C61A8448499
:1066F0004E7038066DA0860DA40C570C470E5E5ADE
:10670000A84EE88BF59C0E1CA2B86190AEC6E8B806
:106710001CAAAEA8A0844D90CC01B27CC6BCE83DBA
:10672000AC91A44EF0688DACAE5891A49828F94075
:106730004E6828DAE59A353838054070066666787E
:10674000F0EE0D107D88EE70E9907C2370E990A644
:106750006DA4AEE89DA4840C270C2F084CB1223008
:10676000BD02CEBEEECEBEEECEBEEEE044840DA4A3
:106770000E1C0A3003E6F86190E6A0F6DF06261F3D
:1067800088B348A36601A4BEBAB06544848DAC1931
:10679000AC19AC700DA4EECE61901CCAA8A9A43CA3
:1067A000E091A4B0FA274626765C5A5E50EE4E1C65
:1067B00098163C422666E21B4213A6566F58860680
:1067C00046B6504626561B26986E46E09DA44EF0CF
:1067D0005D90B0A8AEA85C4E90E8A9A45E46F0918A
:1067E000A44E68E8380EB8FD4068380E78F5407859
:1067F0008D383D40844E22E80EF8F540FEFD97F8B6
:10680000853C718028F80EFD40F80540388D38F839
:10681000853C4E669041387038ED40B08D38700E32
:1068200038FD40F0ED4028066648CD925D90AEA858
:1068300038F02806669B0E46E8E0B0A0A6A6A1B3F5
:10684000A645B7A60997A62F5D90B8FD40A8F80EFB
:10685000F87D3C718085404EBE504138794091A40E
:10686000B88D38F80540E8380E78F01138B0FED809
:10687000A9A4FED80D407940A9A4A6F07E91A4CE8B
:10688000684E900EF8FD40B596F81D3868F80EF881
:106890007D3CF0B80E787D3CB8D940B00540353825
:1068A000B80540A84D409DA47091A4F8853CB8D986
:1068B00040B0554091A4B80EF0FD4078853C614051
:1068C0006184554091A4B870F8FA23DA50260EE896
:1068D0008538854085A4B0AE7D3CB00540A8619C5C
:1068E0002E7A553C6D40709E91A4CE68A9A4A60650
:1068F000F0B0D94058388DA4AEE89828B80EB0F55D
:106900004068B0A888084EA8F84AFC0E4E1C50E813
:10691000901C029C48021BAE44F08C1F041384B8E8
:106920000E4E5C1085384ED00540A8380EF87038F1
:10693000F94091A4780540E8B80EE0DCA01CF252C2
:106940005E1B6692F85EF940FE238408F80EB09C48
:1069500002D3AE70AE38BEAE227038FD4091A4B8FE
:106960008D38F8853C4E90D940FE1B8808380EF8CB
:1069700070AEF091A4F80EB87D3C38054028F80EB2
:106980000CCBB0AE9C22E802419AF80E4C3738AEE0
:1069900070AEF0A9A43E4D967EEF3885A47819AC70
:1069A000F54091A4B870389D88980EB01138704D9C
:1069B000401E91A4B88D38B0FA435A5E5066D41484
:1069C000EB35408DACB001401D9CEE559304041591
:1069D000322E44601C0DA4EA0EF861901CE21F04E4
:1069E0001322E89DA4AE1CEAA8F8E005A8452409F6
:1069F0009CB8F61F1CD0061CD0B656F6A678FD9C97
:106A0000B806FD9CEE7C5CD0231C6124E61F7ECE84
:106A1000BC76FABCFAE08C2788A922849502F85C3F
:106A2000A2E8D38C27B07EFEE1025E7E0E45543D87
:106A30004CE5368CA70C75CE21BCF05845BC4554AE
:106A400098706B0C1F0CA030107038A0266028F8CE
:106A5000E633DDA4229D9D301070B806F866BF387D
:106A600029A446E33D9CE6A03D9CE6B3DDA42201BB
:106A7000A7301070F81CE65316D0164BB636DCF073
:106A8000E030FFDB661C50BB0DA45B79A4F1A4E6EB
:106A9000A7B806F8A6E89DA47376F6371CD02A138B
:106AA00046F3EE0C8311BCAE09BCAEF001BCAEF0F7
:106AB00021BCAEF059A40E7828B868EEE0EEB30E13
:106AC0007D88AEE00000000000000E5C62E04ED861
:106AD00061A0EECEE0FC5C34CC7460A0494CCC608C
:106AE00060005C4ED01050D050105090D0D050D09C
:106AF000505CE0F8448460FEFE2BFE174888A05CE2
:106B0000B0F9820C5F0C4FC1CCA18C4554E14CEE26
:106B10004E70DCD010901010D01010684E5C101029
:106B2000D010D01090A8EE30E00C1720608C60F9E7
:106B30001004881A1EBA4EE01D4498D44AFA1BE687
:106B4000FEE0AED8601E1A3A79A4FE8B4E4651A2E2
:106B50009CB6FC1A7C1EBE66660676CB2213BA363D
:106B600013BA7C2213BA3613BA7C2213BA3613BA7C
:106B70007C2213BAA666067038261363E62B5A7C6D
:106B80000E66072213BA3CBEDB4EA6A65606E606E4
:106B9000E606BC1A3C0681CC605EFADABC0E79A42B
:106BA00031A45CAAE060660DA4E6C12E5A5C50FADE
:106BB0007658F8761CEA1F30FF1A0698DC901C6A9B
:106BC0001F883CBE9EA6065670381BBE3CB6EB66C0
:106BD0006A833CBEE3661A8C334C874884D3A6167E
:106BE000DB3ED31A3A9F565F7E9E7EBEBCF666841D
:106BF0004430107038DCD08B56CB7E6B3A4B569BB2
:106C000066661CD01653A06660283017AB3016930A
:106C1000301A1C73469BAEAEAEC65E6B30151B0EB3
:106C20004E7038E00E3010D33014BB8DAC0E308077
:106C30008B30907330035B30814330822B0E308376
:106C40000B9C06567038B6133CB6F3E0FAA00E8ED5
:106C50002626065C4647D4941BCEE066D34EDA8CDB
:106C600093DCD423B51C2BDCB51CD4D4B51C0ECEC0
:106C7000E13A0EAD1CDCD417DCAD1CEE4EEE93EA0F
:106C8000EA8E8E7388AEDCD4BBCE667038AEFC1C48
:106C90000ADC7CAEF073B1A80DA45AFCC658F8E625
:106CA000A922769C1BDCDC76EB5670EE3822B7DC32
:106CB000AEEAEA8E8E986E9C8CA35C93A6AE0E70A4
:106CC000383C8C133CAE6A2670AEF0A6986677AE60
:106CD00070EEBA5A3B8C2BBA5A174EF00DA43D9C5D
:106CE0008C3D9D059C91CC8495025C44E616864BB8
:106CF00089A888E05C0644448484C4C4E00C600530
:106D0000A849A47C5606307BC6A6D349A460448417
:106D10007C061C30806AA089908C2F4C374633301B
:106D2000171B3005064E3008581A7A8E2B0EFC16AB
:106D3000AE583C75ACBA3CE61C4A23CA1F06264234
:106D400033C223DC154E4EC6BC1A8EE6EEEE98BA60
:106D500058CE0E3A462635CC7CC92CC65ABCA6065F
:106D6000BC1A6E983CFE78C92C0EB8C92C26A60613
:106D70009F6E78EE4EA606561C3B6E4A7CDCDC6E9F
:106D80007ECB6E78C92CE6AE68B86EEE983C1EDC01
:106D9000901ECF7EFC5C7E67FCDC7E47EE78EE9C2E
:106DA0003C7E93EAD4D4D4D4EACEF0AEE63CA63C02
:106DB000A6ADAC56602E1C336A70EEF0EE6AD7E0DA
:106DC00019A4E2674B65440E4CBFB019AC0D10AE70
:106DD000A15C5C0CA021BCD801BCD8F009BCD8F0E7
:106DE00011BCD8F059A619A45CE2D310BB0D100B4E
:106DF0005821BC619CEE98A80C3B11BCEEF04E7083
:106E0000AEE0B00C730E21BC5801BCD8F021BCD848
:106E1000F0AE3DACF05BCDAC43AE4E70381BB07CF9
:106E20009C62A03CA28DA8412C06983C512CC6E641
:106E30007CC92CA666E6F1BE5A3C66C646BC1AF66C
:106E40009F86465BEE6670EE38AE6670AEF0BAAB0B
:106E500066C6E066A68646005BEE2670EE38AE2675
:106E600070AEF0BAAB66C626E039CCEE7026EE38CE
:106E7000F980DC94BB5CB02BD4D4D4D4D460301073
:106E800070787C561B26DC54EB70388B4D40DD400F
:106E90003856703860F62BA05676E056A0E098433E
:106EA000B00E4D2CEEAE7C0E3010709CB8603C6283
:106EB0007C62477C622F783C62BB3C5A7CC60E1CCD
:106EC000E0EE5CEA23CE5066EEE0C61CD0BCE89152
:106ED000A44EA8E8B0283DAC4EEEA74E6F91A4BDDD
:106EE000DC9CD08668280609925C621BA2A291A451
:106EF000AE9BEE9785A43819AC43B085A419ACB508
:106F0000A4F084F99A70D1A4EEA9B60EB05EFED5B5
:106F1000B71EF940FE17EEDDB2C1A4EE63A9A45C72
:106F200002D05C620213A2E8D1A4A878283868B025
:106F3000E8F8B9DC3A853879404DB8EE6B554491A4
:106F4000D8BDDC2626D940FE3FBDDC262691D8914F
:106F5000A40E78F54079402D80B5A455406140D805
:106F60005EFECB4D404E3E6E8D387DB8EE5F61408B
:106F7000B5A405407DB8EEB338C1B64D40BDDC3A8E
:106F800043C1A4EE2FB0A89DB2A9A45CE225B662CD
:106F9000E829B87940B0CDA4F9404D40213C794072
:106FA0004DB8794039B8553CBE1EE140A18891A446
:106FB0000E38F540553C3ECE43E14CBE1E1DB81B7D
:106FC000854075B4EE57854075B4EE2738282B38C8
:106FD0004EEE27D1A485A48DACB5A4F01D9CEE2F58
:106FE0001C0C154E8481023538B5A4054065B828BF
:106FF0000E784EE0B0E84EA891A42806480992F811
:10700000A8786DB82884B0E838688DA4F940794034
:10701000C1A40EF87D3CBDDC3AD940553C0EB5A468
:10702000FD407DB8EE2F39B8B5A45CFA37BEB62660
:10703000228B5E37FE373A5BBBFEE762FA1B2213F8
:10704000667A0065B8284EEEC1B2B870388DA44E8D
:10705000EE27B08C5BAE0E0666C9B6EEA9B270CD57
:10706000A45EFED5B7F8AE7D3C8540794091A40E74
:1070700038F9402938794029B85544B9DCF9406DD0
:10708000B8A8EDB4F940FE1BC1A45EA8EDB4FD4064
:107090007940C1A4B9DCFD40553C7940F1B486D9B2
:1070A00041FEEB4D40B0BE8D3983C1A4EDB486F9ED
:1070B00041FE6BC1A40EB0213865B8A888F1B6B006
:1070C000262626BEAF0EBDDC666666E07910A00DF2
:1070D000428540DB91A4381B91A40E782BC1A40EED
:1070E000F8F94265448DA4AEE065B80E28784EE00C
:1070F000E6461CA2E6E6E6C6029CE24B300A9C028B
:107100001F881376E6E0301246865CC4C61DAC0EBE
:10711000B0E0481C02300AB68CB70A23F6134A3096
:1071200002C62749A47C56467CC92C0675CEDB30A6
:1071300012A69C2222A7998C9437B9A0D1B80B1A19
:10714000AE5859A44C6DA4FA23F617EEB04C17783C
:10715000F6DFFACBD1B89A9A981A58CE8ED1B89851
:107160001A58AE5ABCFA51AC3A1F260F986E263701
:10717000363A1736586ECE35CC9816860CC70CB7F3
:107180003C5C4A6ADCD09CD0E217D00E1CE217EAC5
:10719000664554E14C9C09BA6DA478A076B66FB6EA
:1071A0009F0C1F0C13C479B884CD3C01A01EFD4078
:1071B000F06DA679B8B3F6134E066606E5AB7EFE13
:1071C00005825E66601ADC0AF62B9A02FC53E68999
:1071D000BB7CE606E6E64646FC46E084B07EFEA1C1
:1071E0008E3EEE8C6084049C981CE2330862E213AD
:1071F0008860069CA24670300A061706A0CE660C70
:107200003756B7301006D326061F6606658CF61370
:10721000DC6DBC281E56074B66866646874E3E13BD
:10722000B0280861BC2361BC288CF7F623A08676C1
:10723000A69CEAEAEA73FE1FFA4B8E26F32B7EA683
:1072400046EF608438DE06E0E676A63030C6FB46C0
:10725000C6C6FB46C65C13A2A6977EA066D4606233
:10726000BBBB66658C0E0A5A137E0ABEBAFE930C2F
:10727000BB26F64B76F62FB00E1E5B36A6CEA606C4
:107280001E1A60AA06A0E026D49BDC435C331C23B4
:107290009C139C3010707830097C366066DC54EBAF
:1072A000F617A0565DA65A9C90102B5A5CD0D0FCC5
:1072B00030F65A56E0F59C0E1CA2B8619066AEE816
:1072C000B81CAAAEA8BD02000000D4CCE23A2EC57C
:1072D000D4AEEE8E4C2B8CFDC3AE44841B4C3B8C49
:1072E00001C3AE4813444488BB4C2B8C69C3AE48E1
:1072F00084734C438C99D7447CA9C6EEA13E485870
:10730000A9A45CA2E8E5A0F80E986E19DC6EFDDC7D
:10731000AE55ACFDDCD5C06A173CC9DCAE281DAC4F
:10732000AE4C5F8C334C13AEBE00FD40438C2785C2
:10733000381B7D3C3D4081C47CF3C1CC45027C516F
:107340002C7C0A3C56CA7CAAE0446E71ACEE71AC4F
:107350006E5C85D4EDDC55A47C9C6251AD59A4D102
:10736000C07C0E492CAEAA3CF9DC512CAEAA3C6A7A
:10737000C1C315DC0E1DACAE3C581DACD83C5670DC
:10738000984CF5192D40C9DC1C2A3C2A3C26034C9C
:107390007B8C6B8483E6E63C56FEA00DC8134C8DB7
:1073A000D68CEB447C58BA5DD4A6D8629BD875AC19
:1073B000FCC68C2F7CA6FCA6D875AC98FCA6587C85
:1073C00079D44C5FFDDC75AC986AAF3C79D4EDDCC8
:1073D000D819DC063CE6B9A8412CC9DC7C1CAAFC07
:1073E00055A44D2CAA492CAEFCAAFC06668C170AA3
:1073F0006AC1C37CEACAFCEA6A07FCEE7E79401CDB
:107400007EEEAA41DC09AC4C27F1CC134E35404D41
:10741000407EEE8DC47C2A7C033C6A0A3CEDC006AB
:10742000667C8C130A7C0A7C6A3B467038601C2A96
:10743000E08445D475AC3C85D4EDDC0E51ACC1CCB8
:1074400029DCCC2701D0688C9739CCB1D0C1CC4C89
:1074500025C755A4488401C288CBBDDCCD8CA1884A
:10746000C9DC163CB6765FFC68CDDCC9DC3CDE3C92
:107470005EA04D40D8FEF1CD781DAC8D381C107645
:1074800027B60AAA36761F760AA188786079DC3C8E
:10749000AB593C0E65026DA4BDDCF0688102300E74
:1074A00058A0B9A8300906986666B78B45D4CDCCEC
:1074B000C5CC0DC851ACE62DC0CDCCC9DC063CC650
:1074C00091AC51ACEEEEEEDAC6E6C6BCC9DCBA1A37
:1074D0009C0A26FB70EE38AE70D83845DCAEF0EE74
:1074E00070D8AEF0D86626BA63661A0A3C4666467D
:1074F000BCC67C661F3C8BB045D40DC88102447C61
:107500005871C8CBC48845D40DC8D5CC7371C84157
:107510002C0A3CAA3CEE51ACEA5B3CEEAA3CEA3CAD
:107520002A0A7C6AE315DC85DCCC973836F031DC3E
:10753000781C0A3CCA3C4A7CAA0AFC0A2FCA7C2A4C
:10754000BB3CEACA7C0A7C4A7C6A1F2AEB7CAA689C
:107550000EB8AE85DC3836AEF0AECC9BC9DC1C0B69
:1075600051ACE63C29CC98D5C06A603C0E1DAC4CB1
:1075700045DCF060AE2A7C937D884CC315A059ACE5
:10758000467CA6BCEE704E7028EEEB701DAC5E051E
:107590004060B0267AB3707940614009B8604D40D0
:1075A000D8FEC989DD4078663F680EB0BA2E3359DF
:1075B0003C6D02F59CB05ED37D884CC315A08DD880
:1075C000B0D1C06A7715DC1DAC0E85DCC9DC1C2A85
:1075D0007C934D40A0993CD3C9DC5E5A3C3616FCE6
:1075E00016A358CDDCFE983C16FCDCB65623D4AE70
:1075F000DBC279DC43C9DCBEBA68E0881384C459B5
:10760000AC3CE68C2DC1EE3CA63CC619DC7CCC2BF8
:10761000E68C2DC006B9AA3C660613A6BC668E068B
:1076200013267AF3412C46E02679A429A42301A449
:10763000E60DA45E5AA84EE6E8E0B80E60F8619048
:107640001CE21322E89DA45C8A8A8AAEA8AEE0B14F
:1076500020F8E637300CE8E6E6C8CC2366E3E049DC
:107660004CB14E301070F86006E6A01CD076175C66
:10767000E5A4FC16FC366B54277CB6E0A6065666DD
:107680007038C3763C56E0B0BE0E4E5CD0FD40FE76
:107690008541B9A0FE134EE049A4607C0616867CA5
:1076A000A61CCA30060AA01C154E4EDC90A01AEE8D
:1076B0007ABA1A7E60FAFAFAFAAB301070B87C5ACD
:1076C000463C3EE08CA0BEBEBEE0C9DC42F5DC36E6
:1076D000605C42FC1C5050507CB9DC367F11D8C92C
:1076E000DCFC5AAB0617A67683A67302A242E35CC3
:1076F00090681C509C55DC41DC02170241DC62356D
:10770000D8B815D801D8ADDC36439C55DC55DC1112
:10771000D82DDC78B9DC36B711D8DC50DDDCA0FD23
:1077200040FE8BF8FC1DAC2DDC7851DC433C16FC94
:10773000B63C681E7C7E4B781C02A241DC21D878C6
:1077400061D831DCA0FA6778767647FCB9DC1C2278
:1077500046A8B8C9DC58B6167EF63B7E3FFE1FB67B
:107760001BBC56AE09D898D9DC360DD311D8DDDC58
:10777000A07D3CADDCA3C9DCF6A05C42B9DC36E7F9
:1077800039DC68EDDC36B7683DDC6251DC2235D887
:1077900035D861400D4045DC01D84B163CB67C39EC
:1077A000DC6841D8013CBDDC62E2AB683C16767C0B
:1077B000B63C163C2DD8B861D8BEC1D5A9DC535C07
:1077C00062E2EF9C505C50685C02EE9C02533C16F7
:1077D0007CB6FC25D84E4351DC2225D835D86140F3
:1077E00011B8A9DCB9DC7636FFF5DC36CB163CB631
:1077F000BC68C9DC62E2A0E5D862D368028E8E1C48
:10780000A20E5CA21CA28EB5DC3CB616763CB5DCA2
:1078100095D86E1C62EF85DC7C0AB34C8B7C5815C6
:10782000A27CF9DC9C623BE08E8E8E6AA09C154E99
:1078300071AC3C66CF7CF659A471AC3CF687FC7603
:107840007667B05DD4EDDC55A455ACB029DCCC37FF
:1078500001D068B02839CCC1CC5DAC7CEAC9DC1C55
:10786000AA7CA6FC289C107C16FC369616BC364BCF
:1078700068E5D86221D97883385C507CF5DC369F86
:10788000FC1C1050285C3DDC629C50D9D409DC2AD9
:10789000A353163CB6F6C1C21C1050BC287C167C03
:1078A000B6FC16763CB6BCD9D47940787CC461D895
:1078B000C8C1D409DC2A33BC76E3CD8CDD40213E3F
:1078C00079D878BC06BCA6FC85D8614009BA680E98
:1078D000BA3C5CA2BC9C9BB813680EBA5CA2EE5C7E
:1078E000A2539C025A3CA2027CA23C607C06FCA6ED
:1078F00016060E8E865C02A2A21F06EB56CC3B65D6
:10790000DCA67CE8FC70380E29AE654465DC70AE00
:10791000F0E30E5CA29CA25DDCA65C5DDCA01CE03A
:107920001C727CA695D8722F267C26CBA059A6FC6B
:10793000EECE1DAC0ECE7C1DACAEF0C65670AEF0D9
:10794000CE60E00E8E9CA27CA21FFCEB5CE2EE02FD
:10795000EE9CE0167CB6FC600EBC5C028DDB3C1C31
:10796000A25CA29CA286A665DC8EAE145F7C1CA6DF
:10797000A626AAFC0A1C7BB5DC3C02BC4255A4F836
:107980007CA63CE8F8FC8EB68E8E861CAA7CE88D20
:10799000D8F87C1DAC65DC7DDCF8FC7659A7267C2C
:1079A000E8F87C81DCBCE85B3C163C16234E318E4B
:1079B0001C7C6A763C769C7C168686621F06EBBC35
:1079C000167CB681DC7C16FC56FC9C0E8E86621FF3
:1079D00006EBBC0646BC16063C267C19DC8DD8B8E6
:1079E0000E1DACAE7C7DDCB81C7C6AEAA03CA9DC38
:1079F0007C9DDCA86301D878603C36167C9616E046
:107A00003C16FCB6B3C9DC3C3616BC9301D838BC76
:107A10008DC40A7C8A0A7CE05C02EEDCA2E05C0297
:107A20008ED4D30E4670F8FCE01DAC85384D400D69
:107A300040A18863EE7841D8EE6544F055A4789C67
:107A4000FB55A4B8DBE5A0C80E301070B8BC8B3C69
:107A500055A4AE685B5E55A4AEA82BEE1BA0BE601D
:107A6000E08EAEA6A26026EB1C2A068686601C0A63
:107A7000E0067CD306FCBBAEA6A626A6E056703870
:107A80000E5E60F6631C1076333656F6333C3E1BB2
:107A9000B63C3EE05DACE67A3C6AE7FCAA7C0E466A
:107AA00070AE680A2A6AAA7677F663567038C8F606
:107AB00033A0B660F660C4E00E4E5C22E000000029
:107AC000000000000000000000000304050A080692
:107AD0000BFF0209070D010C00FF20256920256915
:107AE0002025692D256900202025633A256900207D
:107AF0002020205F5F7C002C0044697370206F663B
:107B0000660D0A005553455200460047004245475E
:107B1000494E0052414400442E4D59005052474DA9
:107B20000055534552202020006620200067202069
:107B300000424547494E2020202020005241442049
:107B4000202000442E4D59202020004320202000DA
:107B5000033E000000000000610D00001B3E00001D
:107B6000203E00001E3E0000FF000000B90600009D
:107B70002A3E0000343E0000933700000000000061
:107B8000A5040000463E0000203E0000523E0000DA
:107B900000000000B1050000543E0000203E00003F
:107BA000603E00000000000011070000623E00007F
:107BB000203E00000F000000F4010000040103015A
:107BC0000201010411040F0417041601180100003A
:107BD000217B0000297B00002D7B0000317B000011
:107BE0000B7B00003C7B0000437B00004B7B0000D4
:107BF0001C7B000000171B243E42536975050205DB
:107C00000804080B08040405010504090809040612
:107C1000080702060204020601060407010308031E
:107C2000040C080D020C0203020C010C040D010DE2
:107C3000080D0408020808070802020704080108E2
:107C400004090209010A080B020A0201080A010AD2
:107C5000040B01020802041008110210021108109E
:107C60000110041101120212011302130812080F6D
:107C70000812041301130414021401150215081448
:107C80000817081404150115041702170119081A1A
:107C90000219021602190119041A01160816041B0A
:107CA000021B081A0818021A041B011B04180818E2
:107CB000040B042020202020202020202000000071
:107CC00001000000047B0000097B00000B7B00002A
:107CD0000D7B00000B7B0000137B0000177B000076
:087CE0007F3700001C7B00004F
:040000030000353193
:00000001FF
